:04080000BAEF57F004
:08080800046ED8CF05F0E0CF2B
:1008100006F00001E9CF0CF0EACF07F0E1CF08F0D5
:10082000E2CF09F0D9CF0AF0DACF0BF0F3CF12F014
:10083000F4CF13F0FACF14F0F5CF15F0F6CF16F091
:10084000F7CF17F000C00EF001C00FF002C010F09B
:1008500003C011F0F2AA30EF04F0F2B46BEF1FF016
:100860000EC000F00FC001F010C002F011C003F084
:100870000CC0E9FF07C0EAFF078E08C0E1FF09C00E
:10088000E2FF0AC0D9FF0BC0DAFF12C0F3FF13C0AA
:10089000F4FF14C0FAFF15C0F5FF16C0F6FF17C02D
:1008A000F7FF045006C0E0FF05C0D8FF1000F76A4C
:1008B000BE0FF66E080EF7220900F5501200000177
:1008C00002030405060715161718191A1C1D1E1F0A
:1008D00020212223262B2C2D2E2F3031323334355C
:1008E00036373A3F4041424344454647A2131091B0
:1008F00000010515A00000023402FFFFFFFFAA550A
:10090000AA5503000000000000000011AA55AA55D6
:1009100003000000000000000011280FF66E090E11
:10092000F7220900F550120008090A0B11121314DE
:10093000909192939495969798999A9BF0F1F2F3EF
:10094000F4F5F6F7F8F9FAFBFEFF5C5A09F9EA84C8
:100950001B67498B33AC72C64A1990E91BE64F2BD3
:1009600003AEA92DB39C9123CC6DAFAFE429ECE18C
:100970002462F293848637A7B4B142106534679637
:10098000F912F292700E4E088EBBEE9EAFAF660566
:100990004194DAE54AE4DEF423A944D40EE6CCD54A
:1009A0009122EE6260FE500617EF50B2BC61AFAF0D
:1009B0003FEF6282A31EF58430333368AD1ECCA7AF
:1009C0006DC3B479D76C6E7CA7CFB750F0DBDFF581
:1009D000AFAF212B9BA8BCADF5A30ADA368F3375D8
:1009E0009A8B896A741C43B5C5643AFF742610114A
:1009F0007855AFAFA035458AA1CBEF7C419BEBF09A
:100A0000340A918AD750326B583A1C4EFE348FB953
:100A100002EB056AAFAFA0910C3EF82B6CD9210414
:100A2000B5DC39F04082BC5441C3C58B6DC271DF67
:100A300035A65B2F4219AFAFA0910C3EF82B6CD9B5
:100A40002104B5DC39F04082BC5441C3C58B6DC272
:100A500071DF35A65B2F4219AFAF20DE7802712C13
:100A60008C0F8B1C4EF9E6C51C4B801149E6CD6AF4
:100A70004AFA911F7671EAA8BA11AFAFD3BC913F81
:100A8000102532236730AD31B41C744C37AD6EB1D4
:100A9000647BF7EDAFE9049E8D8DC1A5AFAF2FB399
:100AA00036CD7BED291B8222419D8E0A79FC446D57
:100AB00090EA7CB369C5B2EBAD5CA68ADAF6AFAF5B
:100AC0006044CA33237ECBBD59BC35BA64901CC385
:100AD000EC97BB03CBCBF6552C699B740BF44DFA0A
:100AE000AFAF9864818C5A19D4EF0E654980C477F2
:100AF000A615500EE30CA5F3E1032479F079E88EF6
:100B0000B9F2AFAF3CB171C5BFE2D8ED8DA09F7B0C
:100B10008761B79FD4A85316989C7707CCE5E385E7
:100B2000E1E77301AFAFF4BDA253D2F5482349EA20
:100B300086B0710D6055AD269DAFA6C7D6152C4663
:100B4000833279258BD0AFAF0260CB952C10606ECD
:100B500003A786E74A60C1E470FF566F47AF1F7175
:100B6000387DC1246BCC5FDAAFAFD48B471F7D38A3
:100B70005FFA17E62E7E7F2EC968289A07B56E03A6
:100B8000100B99D68A23AD95FACDAFAF88FF30F11F
:100B90005F32D6E3630470B2AB308A4A7DC5967289
:100BA000C811DE8FA9C8BED58E7243D8AFAF2362FD
:100BB000AB5A770A08D136EFB1DB3CB93082E88313
:100BC00060B80E171AAD71074377E757FE5AAFAFFB
:100BD000E62A48695ACDF723F33CEA0540C947B8ED
:100BE000ADFFDF781BB199FDDC8A46F596F54742EB
:100BF000AFAFDC3E4F3707A7995ACC4569405F0538
:100C0000526343932F7977BF8DB03F2ACF4C0502B3
:100C10000F87AFAF6A831E9A0DE61F3528EB5F87FB
:100C20007BFF5ABA3CD4CA510F2A9F0D2366C3B129
:100C3000FCD5F54CAFAF0E4D1FE241C5A2CFF62358
:100C40004C4B3F11BB8CC2FB51A5B270679F540C3B
:100C5000FB6ABDA15694AFAFF766F846C6891C5033
:100C60002AADBB8F1BCDBC112BDB58A2177F940E76
:100C7000E430D00286B66507AFAFB5C279DA188A1C
:100C800002590DB73CF23DC7BDF68358B82EB717D1
:100C9000443ABB1DD9FEDE94C2E7AFAFC2BDADD3AF
:100CA000279EA783190223B5AB9C873BD74DED0B3D
:100CB0008F1932A08BF0244F25942A1AAFAF8A5A8D
:100CC0007C5353192E2A5B472FD1D5A3DE223CBF7C
:100CD0006A7E813BF5A54A38D7590103E08CAFAF56
:100CE00064359AAFBF49A2C5EB498DBDAAEFB1B338
:100CF00076AF61458127EE14D5625970B2F947612C
:100D0000AFAF6EE27E22D578AD3AE4916056955B46
:100D1000D968EA649C9C08D670533FDEBBDBE7E1F0
:100D2000F7AFAFAF73F23CF116EB5ABC9A474AB833
:100D3000C16A13380B9A8C5FE70CE8E37D36FCB38D
:100D400029092F624F4FCCD921ED82965DAFE24C3D
:100D50007640A78ADAC20FDD2B773A5E56276BCA38
:100D6000D61DE29DCC75AFAF6CE177399320834BF4
:100D7000D0938C51638F9210C756BC5A906BD6B4E7
:100D80004B560936130556DCAFAF8B7AE170BAC10A
:100D9000B78EA30908C5B31744E16CB7D921988170
:100DA00071FD2F43BF287081DA71AFAF8205A49621
:100DB0005329B6F9BF1EE3AC5EF7571E9A2022985E
:100DC000359FE525DD4690A120AEFEC1AFAF23A043
:100DD0006B9B1F36FB4D92358385D8ABC6D4D7A904
:100DE00006D0EB098FB765AB514BCF68D1E3AFAFFE
:100DF0002765317AB2B455E669BDFC2E0FFDD9F3F3
:100E0000448D584995B19B1205705BDF160D2A1968
:100E1000AFAF96488EBC12A04959AAD48D638AA15F
:100E20005D00C6D06541BFF82511258F6A59E58B55
:100E3000BD1A4F4F7E1511E3F7990D041D8F0ED685
:100E40002271F39B6702105D0579F3AB59CEEAA7D7
:100E5000D08EF2264F4F99368125D933AD68E4CF35
:100E6000D1D54054F4570B43F837792F8D1840955E
:100E7000CD7C86726D81B0B03E8748B8FC4CAFFF28
:100E80001729884DDD74C58A5DB1C5BB677C22D446
:100E900087C2877CD5C954AFB0B09C7DDF4A1E9015
:100EA000E577B0DB2526ED1279321E1DFF33227661
:100EB000FE2EB4F66F00FD54E20FB0B0CC48000730
:100EC0001A8FCAC9AF78DDA4085F5D5105E9739533
:100ED0006A1FDDE943F6CBC67A08AC6AB0B0E01F02
:100EE000C95824AF34AEDCC1A2D81B54C6A1644893
:100EF000722EB2543AE2E7976458DAA74621B0B0AE
:100F0000F2248ECECEE8062E5EC4384131CDF6E214
:100F1000B8721299681032F475679B447E1020F9FC
:100F2000B0B0B33648BA8F23B78D622883114E050F
:100F300051FF74F7ED5FFE21172A9C4AEE7297FB72
:100F4000A592B0B0D68344C631009869A0AF26FB05
:100F50006611476F4949760AB7167B1325DB59D3CB
:100F60006CD49D3DB0B03DA7AFC4ED7ABEF5E4AE04
:100F7000928F62802DB0F838AEFF62EF3C370A18CE
:100F800086A5B8B6A384B0B04E03500F746A5C480F
:100F9000CDDEE8AFA53EAAE3CD04AAAE98B4BEBEAE
:100FA00026F96CD1FD5DEEFAB1B144191A4409E796
:100FB00053C070328CA0025FF02C6854B99020A707
:100FC00092504B036C13AC62BD77B1B1855A544358
:100FD000D903645250871F3CC617DC15B63AE3AC00
:100FE0008D4694240900039C54A605BFB1B1006C42
:100FF000B4456A1442B970ACE6C70E59059B26BDCC
:1010000018CED5E963B7E83ED2BB3998D598B1B1CF
:1010100065A4E7F773F2FE70CD0ABC3FD3BD0AD7D3
:1010200011DDBEBFA3E44692B49703D86C14B22D71
:10103000B1B1B6AD5B6C1016E8D76AA991B108D70B
:10104000D592BF29DBEA5D112613A04DF712A269E4
:10105000C708B1B1719FCE1ACB6A09420F944651AD
:101060005B3F2B587028131005CBB80388C5EE6A78
:101070007D4AAFE1B1B19FC4B73B490F920BB73C7A
:101080003CDF423BC4E9DB7AA5B0531F8BC9310B6F
:1010900092AB5FEDDF7251519A34BFA71A4B70E2E9
:1010A0005457ED085211A83C01E7D3A78D639AE28B
:1010B000CC4FBA8B2AC38F57B1B1763C4661974C5F
:1010C00001524CC90D6DFE2D610C4620F629285A9F
:1010D0001F4547DBD4AF6107EC5DB1B121F17076FC
:1010E0009A063DC333FD8970B5C10C5E3457312972
:1010F0001983BB26B5E0D44B8E7AE009B2B2124C0C
:10110000D106B8917826A86F313A428297F9198CA6
:10111000D7C96ABDECA8F0FD001228E4487CB2B241
:1011200028630EB2333774935266493EC5CD37A457
:10113000D1746A78E94DBFA6C143D3F9BE3789D4CB
:10114000B2B20588D62772B8E0E6F69D3D09198C43
:101150006365DA83E799C9A596C7B9B70EA08A4037
:10116000D898B2B283BB122418B899F1D41F4DF0AD
:101170002C624C6BA5A95DE7F952039E4A17B39EFA
:101180009DEDC08DB2B22E84F19A9998B03A968DA9
:101190009D76C4EF2328893C087C0A77BBBB25CD0C
:1011A000B4074D5D9A93B2B28306DD27B503C68CB2
:1011B000BF40597EA278026684A20FE87CF2E04626
:1011C0002CEA5F9D01427F3CB2B2F76ADA0FF66EFD
:1011D000110EF7220900F550120000010203040568
:1011E000060708090A0B0C0D0E0F20212223262BBF
:1011F0002C2D2E2C2D2E2F30313233343536373ADC
:101200003F40414243444546A2131088460205151B
:101210004F06A00000034901AA55AA55030000008B
:101220000000000000000000FFAA55AA55030000BE
:10123000000000000000440FF66E120EF7220900B5
:10124000F550120048494A4B4C4D4E4F50515253A5
:101250005455565758595A5B05EA1376C5D9796FD4
:101260006F0FD333D3BEA855F6F6B303094C1E82D5
:10127000A8D80587A5F7EFEF7D9B1A53BBF52C6E19
:101280000EFE311B0032ED536528D15ACFDF556178
:1012900016F6BBF5147A430406E6BBF51B698D42CE
:1012A0002B7108D96D4F021116D14AA87DCE1AF9BB
:1012B000BBF52C6CA6EB7F3D84E0FDDB1C135BD4FF
:1012C0002EBEA9B403E0453A86435FEDFE08471BF6
:1012D000277B9C5D3120ECA77B9BDBC6AD007A278A
:1012E0007B9C33BE27AA01AD57ECF4397BAF7580E8
:1012F000CF4E19F854F4BEA8297F5CD5EB00EA293B
:101300007F5CABBE305370A97F5C53E533520275EE
:101310005201F35F014D4A3352024BBE31EC25B30B
:1013200036D13328343821636D5E3F2D4E74BBF5C2
:101330000DB98FF238A639241B6F8B552528FF3E37
:101340006D7B548D1442BBF5391817E3614A640074
:10135000FE391817B9BE307EC7B91817397E3BE57C
:101360004E70D8DD7B7B8B1397BBF50DAEFDE81B74
:101370003B5541E76E3F3E4EACBEA9B41DE2254051
:10138000A65AB9DF3D34F1B9CDCE3D34F18FBE312F
:1013900023C4BD34F137BD273FE3939193036154D8
:1013A000005A3FE3935BBE310B2BBFE3406A5C1FE7
:1013B000723900FA406A5BF5BE3120EFC06A5B9D6E
:1013C000463D6585ED4A4F8A03E4BEA9B5F6CE0ECB
:1013D0007F0B4A6E49223AF3223A6189A200CE4934
:1013E000223AC9BE31E7B7C9493F3559C7C93F3469
:1013F000D7B623006E493F352FBE315A495DC137FC
:10140000004A495DC103BE314628C95DC0ABF2B296
:101410004977AF61DF20DB007E4977AF37BE329E70
:10142000F6C977AE4A27724D7863A6BEA85786DF05
:101430003036FED431CF7F1E4FA78BC13F8249008B
:10144000DE4FA78B97BE318F43CFA78B506B06C360
:10145000552EF4CD844DFF5E70348BBF6176518E76
:1014600050971F071E85261300DA50971EDDBE31E8
:101470008EC3D09754492A534929D19C1F006E54DA
:10148000492A29BE32A559D454FA2AE3FA2A6120FE
:101490006200FE54FA2AB9BE329655D4562CDC139B
:1014A000827C00EE562CDBE9BE3146BED62CDB91A9
:1014B000581B3B8F3B03E851006A581B3B65BE310C
:1014C0002A93D81B59370A5F3709D73AFD006E595E
:1014D000370A2FBE31EA44D959929E07D9929D8589
:1014E000AE9A00DA59929DDDBE31C40559F2BC9323
:1014F000BE31462AD9F2BC1114A5006E59F2BC695E
:101500005A46AA4146A9BF7A96005E5A46AA17BE15
:10151000319B88DA5A6B45D9EE5A6B45AFBE312301
:10152000E4DA6B45575EFD005B6279C7DE5B62798A
:1015300097BE3146FEDB62793FD707005D13D129A4
:1015400000FE5D13D0FFBE300432DD13D0A7B07EA5
:101550005D33DB5329BE3043E8DD33DAC552CA00C0
:101560006E5D33DB5D67BB3DBABB4BCD005A5D673B
:10157000BB13BE31919DDD675E5A59697E5E5A5933
:101580003FBE31FC07DE5A58DD338C005E775BBD11
:101590005B93BE3146BFDE775B3B64FB00DA5E7770
:1015A0005E975E855E975E5BBE31E7FCDE975E030D
:1015B000C4DF5D5A5F03B93D9A5EDF03B8BB876B3A
:1015C000005A5F03B913BE315F825EDD825EB3BE37
:1015D000305252DF825E5BE02C00FA5F62572A973E
:1015E000E2572A15A97E006A62572A6DBE329EF123
:1015F000638FF68F638FF665BE31FF04E38FF60DC0
:10160000117C006A63E26017D7C000EA63E25FED15
:10161000BE318EAAE3E25F956403EC2DA786004AF3
:101620006403EC03BE319906E403EBA164BFA1514E
:101630008CE4BFA0CF041A006E64BFA127BE31EFB7
:1016400064CD5CE78500FA64CD5CBDBE311739E43A
:10165000CD5C65EE657E5ADB7E5AB1BE3043E9E56E
:101660007E5A4F3C33EFEE656587855757E5878493
:10167000D540CE006A6587852DBE3296677451FCD1
:10168000CB48A76D67BBF50000817104DBBF295F04
:10169000679A7F7D53BE3154EAE79A7EFB5504007A
:1016A0005A679A7F69B8396996E9B838E72CD0004B
:1016B0007E69B8393FBE313D69DB4B0D4AE3BE312F
:1016C000C5F3E9DB4A8BE5AE00EA69DB6A355227F0
:1016D0006A3551E5BE31D5D9EA35518D9C2B00EAEA
:1016E0006AA1A9B19EF2EAA1A925B46D00CE6AA1B2
:1016F000A987BE326B52ADFD6DEB52AD7BA86A007F
:10170000DA6B52ADD3BE31FF6B88118716EAEB88D6
:1017100011054F91005A6B88115DBE316CB7BA7FCD
:10172000B7B9F30866004A6CB7BA4BBE314155EC05
:101730006CC96365F3BF6172A893E2411418FDFFA1
:10174000EE76C1036D103B973B15C95E006A6D10C4
:101750003B6DBE31173AED106DA2B4DD319479EDD9
:10176000A2B45B51A700FA6DA2B4B3BE6E4571215D
:10177000FDFE6E4570F7BE31C8F5EE45709F924A8A
:101780006F157D794E6F157D49BE314696EF157CFC
:10179000F1D385007230750A6FFA318621DFBEA859
:1017A00055F0F8A00A0FC12473061773F11A11003F
:1017B0004E73061749BE3123CDF306167415B7B51F
:1017C000B7333DFFCDCA7415B78BBE31FF06F41594
:1017D0007531868BF531860956C3005E7531866199
:1017E000BE31BB927645B423BE31DF42F645B39796
:1017F0002DA100FE7645B3F9766EE4F7C600CA76F1
:101800006EE4CDBE31DDD0F66EE4753D769388276B
:10181000BE329A3CF69387A57EC400FA769387FD84
:1018200077679ABDF7679A3B6B3B00DA77679A93C5
:10183000BE3053A2782DFC0B9EB700DE782DFBE165
:10184000BE31BB89F82DFB897969DBF7CDBE3073DA
:10185000C7F969DB75A5C300CA7969DB79E57269E7
:10186000E5723FBE310B22F9E571E7634B007E79EB
:101870007C12635D33BE32A999FC1262D1B7580065
:101880007A7C12637C67D84714005A7C67D81DBEE7
:101890003194F2FC67D7C5BC7CCF17B978CB7F1CDD
:1018A0005F6B71477211BEA9B5F4CC247F0D4F2137
:1018B0004EF7BE328678FF0D4E9FBA0800FE7F0DB0
:1018C0007F8767451BBE31C4C8FF8766C37EC000E3
:1018D0005A7F87677FD6BCD932916CFFD6BC575EE2
:1018E000F100EE7FD6BCAFBE8155B835BE32A82818
:1018F0008155B7B36EC8004A8155B80B8314CF6FBA
:1019000045BE31D5D48314CEED96E2004A8314CF80
:1019100083165CEBFE00FE83165CC1BE31D187836B
:10192000165C6937835361754A8353614BBE31EC52
:1019300062835360F397B900846DA9558C846DA8B8
:10194000C7A3F95D5E846DA91FBE316C84B86E912A
:1019500084B86E67BE3194F384B86E0F334A006E5C
:1019600085D131C37485D13141B25300DE85D13187
:1019700099BE31EC872D146931308D872D13E1C16B
:101980003E7F7E872D1439BE88199B3F9ABDE88D16
:101990004F5A88199B15BE32916D881989D623F745
:1019A0006B9F7FCFCA89D623CDBE31895A89D62372
:1019B0008B500D1DD21E8B500C951C0FEFEA8B50D7
:1019C0000CEDBE318D17C4D54700EA8D17C4ABBEF0
:1019D00032B6578D17C453398FAE86BD8FAE863B56
:1019E000DC8900DA8FAE8693BE3130868FB00E135D
:1019F0008FB00D91BA6A00EE8FB00DE9BE32867AD3
:101A000091B0BAAD91B0BA2B1FB400CA91B0BA83ED
:101A1000BE30076093080FBD0F3B276C00DA9308B8
:101A20000F93BE318EDB93089551784FAF006A95C6
:101A3000517825BE32B650955177C15D95BFDF29EB
:101A4000DEFFBE31A45995BFDEA7B66600FE95BF86
:101A5000981170398D57004E9811700FBE32A8073B
:101A600098116FB7986E8631986E85978CC700EE87
:101A7000986E85EFBE31C4CB9944221799442195C5
:101A8000E21900EA994421EDBE32A5B69C55FC0549
:101A90007FFD00DA9C55FBDBBE31336A9C55FB773A
:101AA0009E48ED4B5E9E48ED21BE3123CA9E48EC18
:101AB000BF0D30009EF9EDCBCE9EF9ED89BE3123EE
:101AC000D89EF9ED310068CF9F864B814B57BE31D0
:101AD000683E9F864AFF10F7005E9F86A05BEF7905
:101AE0004FBE3198AAA05BEEED7382004EA05BEF73
:101AF000A19DE35D33BE32A5B7A19DE2D10B82006B
:101B00007AA19DE3A2C8F605A2C8F5C3BE3189DE5D
:101B1000A2C8F56BE27100CAA3B0E5637AA3B0E591
:101B200033BE319418A3B0E4DBCDA000A549D84F53
:101B300024006AA549D825BE304AB7A549D7CD0F9C
:101B4000A7EC43B14387BE319F8BA7EC432F2F9265
:101B5000CDCEA7ECA85283EB69F97500FEA852839D
:101B6000C1BE31DD2EA85283A93F0285A93F01FDE8
:101B7000D279005AA93F0255BE3188F4A9746A058A
:101B8000A97469DBBE3187F6A9746983DFA300DA23
:101B9000A9AB5A6DAB5A43BE3116FEA9AB59EB2027
:101BA0002F004AA9AC6632B7AC663235E30600CAEC
:101BB000AC66328DBE314699AD820441314141ADB2
:101BC0008203BFF678005EAD820417BEB152913138
:101BD0005AD1B15290AFDAD0004EB1529107BE3116
:101BE000B1A8068FB1A8060D3BF2006AB1A8066540
:101BF000BE312DA5B4A605E7C4B4A60565E34CFF28
:101C0000FAB4A605BDBE31C5B4DE77EFC5BE305807
:101C10000DB4DE776D590000CAB4DE77B5CC83F120
:101C20006F790600CEB5CC83C7BE314142B5CC83B7
:101C3000B77229CF28B772294D7B2400EAB77229E1
:101C4000A5BE329EB7834E91B7834E67BEA8D11909
:101C5000B7834E0FE3196D6EBAAE32BFBAAE323DE6
:101C6000156800DABAAE3295BE32BBC9BBDDD8D733
:101C70004B00EABBDDD8ADBE3198D0BBDDD855B541
:101C8000BE1707C3412EAC00DEBE170799BE314117
:101C900043BE1707BFC7B69FBFC7B605E2DB6F7A63
:101CA000BFC7B675BEA8D11AC23B82453B81C3F6F9
:101CB000D4005AC23B821BBE306AD1C2C6618705BE
:101CC000868394C300DAC66186DBBE31415CC6619F
:101CD000CB5D27A1271FA3FE007ECB5D2777BE31FA
:101CE00035DFCB5DCCE54E7BE54E51BE3198CBCC9C
:101CF000E54DF9E382004ECCD3CABFF573E157003E
:101D0000CAD3CABFCBBE319BEFD3CABFD4E1F9F966
:101D1000CED4E1F9CFBE3198D3D4E1F97725B40020
:101D2000D4EE2F992F17B492006ED4EE2F6FBE31E0
:101D3000C40FD4EEDB7075A1006ADB70756DBE3127
:101D40001707DB7075154066DD38AEF738AE75CD18
:101D5000C600CADD38AECDBE31C408DDE044695BE3
:101D60006EE0446931BE31ECD3E04468D91AF30027
:101D7000E127C2F127C2C7BE3198BAE127C26F6519
:101D8000D100CEE1E7116CA38115007EE7116C79DB
:101D9000BE313363E7116C21EE092F092E87013B19
:101DA00000DEEE092EDFBE328792EE09F03930CB2D
:101DB0003193EEF0393049392B00DEF03930A1BED5
:101DC000F940E68BF940E65BBE313538F940E60371
:101DD00015BC5D5AFE210F5FDDCE9A007AFE210F01
:101DE00035BE313D94FE210E0000000000000000D1
:101DF00000000000000000000000000000000000E3
:101E000000000000000000000000000000000000D2
:101E10002563315D2050726F6772616D20426C6185
:101E2000636B202020202020202020202020202024
:101E3000202020325D2050726F6772616D204379DF
:101E4000616E202020202020202020202020202003
:101E500020202025630D0A002563335D2050726F1A
:101E60006772616D204D6167656E7461202020206E
:101E70002020202020202020202020345D2050728F
:101E80006F6772616D2059656C6C6F772020202020
:101E9000202020202020202020202025630D0A0043
:101EA0002563355D2050726F6772616D204C2F4D38
:101EB0006167656E74612020202020202020202072
:101EC000202020365D2050726F6772616D204C2F8C
:101ED0004379616E202020202020202020202020F7
:101EE00020202025630D0A002563375D2050726F86
:101EF0006772616D20436C65616E696E6720436136
:101F000072747269646765202020202020202020C0
:101F100020202020202020202020202020202020C1
:101F2000202020202020202020202025630D0A00B2
:101F300025633D3D3D3D3D3D3D3D3D3D3D3D3D3DC3
:101F40003D3D3D3D3D3D3D3D3D3D3D3D3D3D3D3DC1
:101F50003D3D3D3D3D3D3D3D3D3D3D3D3D3D3D3DB1
:101F60003D3D3D3D3D3D3D3D3D3D3D3D3D3D3D3DA1
:101F70003D3D3D25630D0A0025634D5D20526561A1
:101F800064204D61696E206D656D6F72792020202F
:101F90002020202020202020202020505D2052655D
:101FA00061642050726F74656374696F6E206D6533
:101FB0006D6F72792020202020202025630D0A00DB
:101FC0002563535D205265616420536563757269B2
:101FD0007479206D656D6F7279202020202020207B
:101FE000202020525D205075726368617365206304
:101FF0007265646974732020202020202020202016
:1020000020202025630D0A002563555D2057726945
:102010007465204D61696E206D656D6F7279283130
:102020002062797465292020202020575D20577276
:102030006974652050726F74656374696F6E206D8A
:10204000656D6F727920202020202025630D0A0005
:102050002563515D205772697465205365637572FD
:10206000697479206D656D6F7279202020202020A1
:10207000202020565D2050534320766572696669A2
:10208000636174696F6E2020202020202020202092
:1020900020202025630D0A002563415D20436F70D9
:1020A0007920746F2054656D706C617465202020F8
:1020B0002020202020202020202020425D20506150
:1020C0007374652066726F6D2054656D706C6174F9
:1020D000652020202020202020202025630D0A00BC
:1020E0002563435D204368616E6765206361727498
:1020F00072696467652073657373696F6E20202051
:10210000202020495D20446961676E6F73746963A4
:10211000206F7074696F6E73202020202020202093
:1021200020202025630D0A0025634E5D2052656145
:10213000642054656D706C617465206D656D6F729F
:102140007920202020202020202020445D20436F63
:1021500070792074657874206461746120746F20D4
:10216000636869702020202020202025630D0A004C
:102170000D0D505343207665726966696361746919
:102180006F6E3A2054686520534C45343434322005
:1021900077696C6C20616C6C6F77202575206D6F92
:1021A000726520756E7375636365737366756C20F5
:1021B00077726974652F732E00000D0A5053432007
:1021C00066726565206269747320696E2074686543
:1021D00020534C4534343432206861732062656585
:1021E0006E2065786365656465642E200D0A0000C5
:1021F0000D0A5752495445206F7065726174696FBA
:102200006E7320617265206E6F206C6F6E676572F1
:1022100020706F737369626C652E20524541442DA6
:102220004F4E4C592063617264004E6F20636869A1
:10223000702F636172642064657465637465642ED5
:1022400020496E7365727420636869702F636172D0
:102250006420746F20636F6E74696E7565004368E7
:1022600069702F436172642064657465637465648A
:102270002E2049443A20413231333130393120283F
:10228000526F636B486F7070657220636F6465296D
:102290002000436869702F4361726420646574652F
:1022A000637465642E2049443A2041323133313021
:1022B0003838202856616C75654A657420636F64F0
:1022C000652920202000436869702F4361726420D3
:1022D0006465746563746564206275742066726FEA
:1022E0006D207769746820696E76616C6964204F2F
:1022F000454D2074616720202000313D3232306D21
:102300006C2020323D3434306D6C2000313D383843
:10231000306D6C2020323D313030306D6C2000004B
:102320002E0D0A4E6F74653A20306D6C2077696C03
:102330006C20636175736520612064656661756CEE
:102340007420636170616369747920746F207365B0
:102350006C65637465642E204D61782E3432393596
:102360006D6C20002E2E2E2E2E70726573732061E0
:102370006E79206B657920746F20636F6E74696E5F
:1023800075652E000D0A4E4F54453A556E70726FAA
:102390007465637465642064617461206D61792083
:1023A0006361757365207468697320636869702060
:1023B0006E6F7420746F2062652061636365707452
:1023C000656420627920746865207072696E746536
:1023D000722E0D0A0A004E4F54453A2050726F7407
:1023E000656374696F6E204D656D6F7279206861E9
:1023F00073206265656E2070726F6772616D6D65C6
:10240000642E0D0A0A000D0A50726F6772616D6DBD
:10241000696E67207468652063686970206D656DFA
:102420006F72793A0D0A0000426C61636B202020C4
:1024300020202020202000004379616E20202020D1
:1024400020202020202000004D6167656E746120EF
:10245000202020202020000059656C6C6F77202000
:1024600020202020202000004C69676874204379D8
:10247000616E2020202000004C69676874204D6147
:1024800067656E7461200000436C65616E696E67FC
:1024900020466C7569640000556E6B6E6F776E2018
:1024A000436F6C6F757200004D75746F68205661D4
:1024B0006C75654A657420285553412900004D7597
:1024C000746F682056616C75654A657420313638C2
:1024D00030202855534129004D75746F682056618E
:1024E0006C75654A65742042756C6B2028555341A4
:1024F00029004D75746F682056616C75654A657466
:102500002028455529004D75746F6820526F636B04
:10251000686F7070657200004D75746F6820526F3F
:10252000636B686F707065722042756C6B004D75DF
:10253000746F6820537069746669726500004D7528
:10254000746F682053706974666972652042756C97
:102550006B004D75746F6820426C697A7A617264A1
:1025600000004D75746F685F426C697A7A617264BD
:102570002042756C6B00416766615F414D363500E6
:10258000416766615F414D36352042756C6B0000D6
:102590005865726F78203832353000005865726F98
:1025A0007820383335302042756C6B004F4345201E
:1025B00039303930202D2045636F536F6C76656E4E
:1025C00074004F43452039303930202D204D696C3F
:1025D00064536F6C76656E7400004F43452039304C
:1025E00039302042756C6B0046756A6946696C6DBE
:1025F000204D696C6420536F6C76656E7420427553
:102600006C6B000046757475726520546563686E66
:102610006F6C6F6769657300536F757468204166EE
:102620007269636100002B2B323732312039373623
:102630002D3538313100202020202020202020205E
:102640007777772E467574757265746563686E6FFB
:102650006C6F676965732E636F2E7A61000050722C
:102660006F74656374696F6E204D656D6F7279204C
:1026700064617461202D20333220626974730D0A05
:1026800000005365637572697479204D656D6F72D2
:1026900079286265666F726520757064617465295A
:1026A000202D20005365637572697479204D656D26
:1026B0006F727928616674657220757064617465E3
:1026C00029202D2000004572726F7221210D0A0011
:1026D000536F6D65206F662074686520666972733C
:1026E00074203332206279746573206F66207468B9
:1026F000697320746172676574206368697020690A
:1027000073206C6F636B656420746F205265616425
:10271000204F6E6C7920736F207468650D0A00007D
:10272000646174612063616E6E6F742062652072F3
:102730006570726F6772616D6D65642E2050726F87
:102740006772616D6D696E6720746869732074616A
:102750007267657420636869702077696C6C2062A9
:10276000652061207761737465206F6620610D0AB2
:1027700000007265736574746572206372656469C4
:10278000742E0D0A0A0054727920616E6F746865A8
:102790007220636172642E0D0A0A00005461726730
:1027A00065747320554944206973206C6F636B65B1
:1027B0006420616E64206D617920626520696E63BA
:1027C0006F72726563742061667465722070726FD7
:1027D0006772616D6D696E672E0D0A0043686563EF
:1027E0006B2074686520666972737420636C617312
:1027F00073696669636174696F6E206F66207468BF
:102800006520554944206166746572207265736560
:102810007474696E672E0D0A0A0020202020202083
:10282000256300002020202030302030312030323D
:1028300020303320303420303520303620303720DF
:102840003038203039203041203042203043203091
:10285000442030452030460D0A0020202020202032
:10286000256320002020202A2A2A2A2047656E6519
:10287000726963204D75746F6820496E6B204368E0
:1028800069702050726F6772616D6D657220566558
:102890007220322E353120436F7079726967687407
:1028A00028432932303130202A2A2A2A0D0A0000F2
:1028B000202020202020202020200000202D205417
:1028C000656C3A002020202020202020202020207D
:1028D00020200000202020202043757272656E7435
:1028E00020536573696F6E3A20000D0A0A536176B2
:1028F00065207468652061626F766520646174612B
:10290000207065726D616E656E746C793F20285918
:102910002F4E292000004465766963652053657257
:1029200069616C204E756D6265723A256C75202D5B
:10293000205265736574206C6F673A25750D0A0A1D
:10294000000028506C65617365204E4F54453A2055
:102950007468652061626F766520696E666F726D5E
:102960006174696F6E206D75737420626520717576
:102970006F746564207768656E2070757263686136
:1029800073696E6720637265646974732E0D0A0043
:102990005468697320696E666F726D6174696F6ED9
:1029A000206973207573656420746F2067656E6598
:1029B000726174652061206B657920746861742090
:1029C00077696C6C2062652073656E742062616348
:1029D0006B20746F20796F752E290D0A0A004372DF
:1029E00065646974732072656D61696E696E673ABA
:1029F00020256C750D0A0A000D0A456E746572205B
:102A0000746865206E756D626572206F66207265F0
:102A10007365742063726564697473206265696E9E
:102A200067207075726368617365643A2D202000B9
:102A30000D0A456E74657220746865203430206319
:102A40006861726163746572206B6579636F646538
:102A500020737570706C69656420627920003A2D6E
:102A6000200D0A000D0A5265736574206372656457
:102A700069747320616D6D656E6465642073756340
:102A80006365737366756C6C792066726F6D202553
:102A90006C7520746F20256C752E00000D0A496E30
:102AA00076616C696420636F64652E002A2A2A2A85
:102AB000000052204520532045205400572052202A
:102AC000492054204520202020502052204F2043D0
:102AD0002045205320530000202020532055204320
:102AE00020432045205320462055204C2A2A2A2ABC
:102AF00000000A0A0D524553455420636F756E74E9
:102B000065722069732061646A75737465642074EA
:102B10006F3A20256C750A0D00000D0A20284E6FB3
:102B200020637265646974732072656D61696E6992
:102B30006E672E20507572636861736520637265DD
:102B4000646974732066726F6D2046542E290D0AD5
:102B5000000043415554494F4E2120596F75206F55
:102B60006E6C79206861766520256C7520637265CE
:102B7000646974002072656D61696E696E672E20EC
:102B800050757263686173652063726564697473FC
:102B90002066726F6D200D0A0000206265666F72FC
:102BA0006520796F75722063726564697473206340
:102BB0006F756E7465722072656163686573207AE3
:102BC00065726F2E000020202020436869702F63FB
:102BD000617264204D656D6F7279206D617020287F
:102BE0003862697420782032353662797465203D08
:102BF00020324B62290D0A000D0A0A4368697020D1
:102C0000636F6C6F75723A2D20000D0A496E6B2050
:102C100043617061636974793A2D2000202020207F
:102C20002020202020202020436170616369747976
:102C30002072656D61696E696E673A2D20000D0A1C
:102C40004F454D2049443A2D20004D75746F682042
:102C5000564A20436C65616E696E672020202020F3
:102C6000202020004D75746F6820526F636B686F71
:102C700070706572207365726965732020004D75F0
:102C8000746F6820564A285553412920736572692C
:102C900065732020202020004D75746F6820564AEF
:102CA00020313638302020202020202020202020D5
:102CB00020004D75746F6820564A284555292073A9
:102CC0006572696573202020202020004D75746F87
:102CD0006820564A203136383020202020202020FD
:102CE0002020202020004D75746F6820564A2062F5
:102CF000756C6B20726566696C6C2020202020004A
:102D000041474641204772616E6420536865727086
:102D1000612020202020202020004F4345203930F2
:102D200039302045636F20536F6C76656E742020B8
:102D3000202020004F43452039303930204D696C28
:102D40006420536F6C76656E7420202020004675D9
:102D50006A69204D696C6420536F6C76656E7420CF
:102D600020202020202020005865726F782D4D757E
:102D7000746F682020202020202020202020202068
:102D80002000556E6B6E6F776E202D20254C5820DD
:102D900020202020202020202020200050726F742E
:102DA000656374696F6E204D656D6F72793A2D2081
:102DB00000004C6F636B207061747465726E2064E8
:102DC000657465637465642E0D0A00005468697348
:102DD00020636869702073686F756C642066756E17
:102DE0006374696F6E004C6F636B207061747465FF
:102DF000726E206E6F742064657465637465642EF2
:102E00000D0A0000546869732063686970206D6161
:102E100079206E6F742066756E6374696F6E000042
:102E20002020202054656D706C617465204D656DA7
:102E30006F7279206D617020283862697420782063
:102E400032353662797465203D20324B62290D0A95
:102E50000A005365637572697479204D656D6F72F0
:102E600079286265666F7265207570646174652982
:102E7000202D20333220626974730D0A00004572E0
:102E8000726F7220436F756E7465723A20000D0A7E
:102E9000416464726573733A200025325820202003
:102EA000446174613A2025325820202056657269A9
:102EB00066793A2000000D0A0A5665726966792023
:102EC0006572726F72206F6E207468652061626F28
:102ED000766520616464726573732E002532582014
:102EE00020202020202020202020202020202020E2
:102EF000202020202020202000000D0A0A50726F80
:102F00006772616D6D696E67207375636365737356
:102F100066756C2E2E2E00004D616B65204528785D
:102F20002961637420636F7079206F7220285229A1
:102F3000656E657720636869703A200020205265CD
:102F40006E657720636F6C6F757220616E642063AD
:102F5000617061636974792073656C6563746F7205
:102F60000D0A000020202D2D2D2D2D2D2D2D2D2D48
:102F70002D2D2D2D2D2D2D2D2D2D2D2D2D2D2D2D81
:102F80002D2D2D2D2D2D2D2D0D0A0A00456E74652C
:102F90007220746865206465736972656420696E67
:102FA0006B20636170616369747920284D617820BA
:102FB000343239346D6C293A20000D0A456E74653F
:102FC0007220746865206465736972656420636F3C
:102FD0006C6F75723A2000000D0A4E4F54453A202E
:102FE00054656D706C6174652064617461207761F3
:102FF000732072656E6577656400536D617274202D
:103000004361726420646174612073617665642039
:10301000746F2074656D706C617465206D656D6F83
:1030200072792E000D0A416464726573733A200050
:10303000253258202020446174613A2025325820DE
:1030400020205665726966793A2000000D0A0A56FA
:103050006572696679206572726F72206F6E207476
:1030600068652061626F7665206164647265737360
:103070002E00253258202020202020202020202013
:103080002020202020202020202020202020000080
:103090004F7065726174696F6E20737563636573D9
:1030A0007366756C2E004F7065726174696F6E2067
:1030B0006E6F74207375636365737366756C2E2011
:1030C00057726974652D25325820526561642D252B
:1030D0003258000020204F454D2053657373696FAF
:1030E0006E2073656C6563746F720D0A000020209A
:1030F0002D2D2D2D2D2D2D2D2D2D2D2D2D2D2D2D00
:103100002D2D2D2D0D0A0A00312E2E2E0000322ECF
:103110002E2E0000482E2E2E0000492E2E2E0000AE
:10312000332E2E2E0000342E2E2E0000352E2E2E65
:103130000000362E2E2E0000372E2E2E0000382EA8
:103140002E2E0000392E2E2E0000412E2E2E000095
:10315000422E2E2E0000432E2E2E0000442E2E2E08
:103160000000452E2E2E0000462E2E2E0000472E4B
:103170002E2E000043686F6F736520616E204F45EF
:103180004D2073657373696F6E2061737369676E29
:103190006D656E742E2E200053657373696F6E20FB
:1031A00073656C65637465643A2D2000456E7465C3
:1031B0007220746865206465736972656420696E45
:1031C0006B20636170616369747920001B0E0400D9
:1031D0009EA8FDD7AD6E5B0E04009EA8FDD7AD6E18
:1031E000320E04009EA8FDD7AD6E4A0E04009EA8C4
:1031F000FDD7AD6E000C0101C351016AC25D03E24F
:10320000C2C100F00CD0006A080EC46FC23700368D
:10321000C351005CD8B0006E0136C42FF7D700014F
:10322000000C0150C0C1C2F1640E0101C36F000166
:10323000E2DF00C0C0F10150300E08E10101C1A37E
:103240000FD0C1B70DD0C1B9200E04D00101C19774
:10325000C199C1810126015004009EA8FDD7AD6E21
:10326000C0C1C2F10A0EC36F0001C5DF00C0C0F1CA
:103270000150300E08E10101C1B70CD0C1A10AD044
:10328000C1B9200E00010126015004009EA8FDD7FF
:10329000AD6E0101300EC027C05104009EA8FDD7BD
:1032A000AD6E0001000C1B0E04009EA8FDD7AD6E94
:1032B0005B0E04009EA8FDD7AD6EBDC1C0F11B0E14
:1032C0000101C16F0001ADDF3B0E04009EA8FDD7D8
:1032D000AD6EBEC1C0F11B0E0101C16F0001A1DFC7
:1032E0003B0E04009EA8FDD7AD6EBFC1C0F11B0E02
:1032F0000101C16F000195DF6D0E04009EA8FDD78E
:10330000AD6E000C0900F5520EE0F6CFBEF1F7CF1E
:10331000BFF1F55004009EA8FDD7AD6EBEC1F6FF0B
:10332000BFC1F7FFEFD7000C1B0E04009EA8FDD70E
:10333000AD6E5B0E04009EA8FDD7AD6E0101C06BA3
:103340001B0EC16F00016DDF3B0E04009EA8FDD770
:10335000AD6E3B0E04009EA8FDD7AD6E6D0E040051
:103360009EA8FDD7AD6E000CD8B204D0010EEA6E57
:10337000D50EE96E006A016A026A036A0101D56B23
:10338000D66BD76BD86BD451D311D211D1112CE09D
:10339000200ED96FD890CD37CE37CF37D037D5372D
:1033A000D637D737D837D451D85D08E1D351D75D58
:1033B00005E1D251D65D02E1D151D55D0FE3D15186
:1033C000D55FD251D8A0D23DD65FD351D8A0D33D3E
:1033D000D75FD451D8A0D43DD85FD880003601360D
:1033E00002360336D92FD6D7D5C1EFFFD6C1ECFFB1
:1033F000D7C1ECFFD8C1ECFF0001000CE95001017E
:10340000C56F3B0ECC6F9A0ECB6FCA0ECA6FC96BDD
:103410000A0EC76FD882010EEA6EC10EE96EC4C1F2
:10342000D0F1C3C1CFF1C2C1CEF1C1C1CDF1CCC188
:10343000D4F1CBC1D3F1CAC1D2F1C9C1D1F10001DC
:1034400093DF0150005213E10101C751010AD8A4D2
:1034500002D000010CD0C5510CE00F0BC75D01E09C
:103460000FE2C5BF0DD0C5BD04D0200E03D00101B1
:10347000C56B300E0026005004009EA8FDD7AD6E2F
:10348000D892CCC1D0F1CBC1CFF1CAC1CEF1C9C164
:10349000CDF1D46BD36BD26B0A0ED16F000164DF18
:1034A00003C0CCF102C0CBF101C0CAF100C0C9F128
:1034B0000101C72FAFD70001000C0900F6CFC0F102
:1034C000F7CFC1F1F55004009EA8FDD7AD6EC0C185
:1034D000F6FFC1C1F7FF0101BF2F01D002D00001EB
:1034E000ECD70001000C1A0EF66E280EF76E060ED1
:1034F0000101BF6F0001E1DFC90E04009EA8FDD7E6
:10350000AD6E0101BE6BBE51330807E3CD0E040062
:103510009EA8FDD7AD6EBE2BF6D7BB0E04009EA8AD
:10352000FDD7AD6E0D0E04009EA8FDD7AD6E0A0E40
:1035300004009EA8FDD7AD6E0001000CDA0E040059
:103540009EA8FDD7AD6EC40E04009EA8FDD7AD6E3B
:10355000C40E04009EA8FDD7AD6EC40E04009EA844
:10356000FDD7AD6EC40E04009EA8FDD7AD6EC40E8F
:1035700004009EA8FDD7AD6ED00E04009EA8FDD716
:10358000AD6E0101BE6BBE51330807E3C40E0400EB
:103590009EA8FDD7AD6EBE2BF6D7D00E04009EA818
:1035A000FDD7AD6EBE6BBE51050807E3C40E040027
:1035B0009EA8FDD7AD6EBE2BF6D7BF0E04009EA809
:1035C000FDD7AD6E0D0E04009EA8FDD7AD6E0A0EA0
:1035D00004009EA8FDD7AD6E0001000CC00E0400D3
:1035E0009EA8FDD7AD6E0101BE6BBE51400807E33A
:1035F000C40E04009EA8FDD7AD6EBE2BF6D7D90E23
:1036000004009EA8FDD7AD6E0D0E04009EA8FDD748
:10361000AD6E0A0E04009EA8FDD7AD6E0001000C31
:1036200062DF5A0EF66E280EF76E060E0101BF6FAE
:10363000000143DFBA0E04009EA8FDD7AD6E200E38
:1036400004009EA8FDD7AD6E01012951006E2A51DC
:10365000036EFF0E035C05E1FF0E005C000112E04B
:103660000101100E035C05E1910E005C00011FE0FA
:103670000101100E035C05E1880E005C00011DE0F5
:10368000010122D0010E0101BD6F938881B808D0DD
:103690002A0EF66E220EF76E000134DE07D001010D
:1036A000C60EF66E220EF76E00012CDE14D05E0EF2
:1036B000F66E220EF76E26DE0ED0920EF66E220EFB
:1036C000F76E20DE08D00101C60EF66E220EF76EF0
:1036D000000118DE00D0BA0E04009EA8FDD7AD6E22
:1036E0000D0E04009EA8FDD7AD6E0A0E04009EA824
:1036F000FDD7AD6E23DFB30E04009EA8FDD7AD6EDF
:10370000120EF66E1E0EF76E410E0101BF6F000124
:10371000D4DEB30E04009EA8FDD7AD6E0D0E0400DE
:103720009EA8FDD7AD6E0A0E04009EA8FDD7AD6E13
:10373000B30E04009EA8FDD7AD6E5A0EF66E1E0E97
:10374000F76E410E0101BF6F0001B7DEB30E04003A
:103750009EA8FDD7AD6E0D0E04009EA8FDD7AD6EE0
:103760000A0E04009EA8FDD7AD6EB30E04009EA8FD
:10377000FDD7AD6EA20EF66E1E0EF76E410E010164
:10378000BF6F00019ADEB30E04009EA8FDD7AD6E98
:103790000D0E04009EA8FDD7AD6E0A0E04009EA873
:1037A000FDD7AD6EB30E04009EA8FDD7AD6EEA0E38
:1037B000F66E1E0EF76E410E0101BF6F00017DDE39
:1037C000B30E04009EA8FDD7AD6E0D0E04009EA89A
:1037D000FDD7AD6E0A0E04009EA8FDD7AD6EB30EE8
:1037E00004009EA8FDD7AD6E320EF66E1F0EF76E6A
:1037F000410E0101BF6F000160DEB30E04009EA800
:10380000FDD7AD6E0D0E04009EA8FDD7AD6E0A0E5D
:1038100004009EA8FDD7AD6EB30E04009EA8FDD790
:10382000AD6E7A0EF66E1F0EF76E410E0101BF6F80
:10383000000143DEB30E04009EA8FDD7AD6E0D0E51
:1038400004009EA8FDD7AD6E0A0E04009EA8FDD709
:10385000AD6EB30E04009EA8FDD7AD6EC20EF66E1F
:103860001F0EF76E410E0101BF6F000126DEB30E81
:1038700004009EA8FDD7AD6E0D0E04009EA8FDD7D6
:10388000AD6E0A0E04009EA8FDD7AD6E1AA057D0EB
:10389000B30E04009EA8FDD7AD6E0A0EF66E200E84
:1038A000F76E410E0101BF6F000107DEB30E040089
:1038B0009EA8FDD7AD6E0D0E04009EA8FDD7AD6E7F
:1038C0000A0E04009EA8FDD7AD6EB30E04009EA89C
:1038D000FDD7AD6E520EF66E200EF76E410E010151
:1038E000BF6F0001EADDB30E04009EA8FDD7AD6EE8
:1038F0000D0E04009EA8FDD7AD6E0A0E04009EA812
:10390000FDD7AD6EB30E04009EA8FDD7AD6E2A0E96
:10391000F66E210EF76E410E0101BF6F0001CDDD85
:10392000B30E04009EA8FDD7AD6E0D0E04009EA838
:10393000FDD7AD6E0A0E04009EA8FDD7AD6EB30E86
:1039400004009EA8FDD7AD6E9A0EF66E200EF76E9F
:10395000410E0101BF6F0001B0DDB30E04009EA84F
:10396000FDD7AD6E0D0E04009EA8FDD7AD6E0A0EFC
:1039700004009EA8FDD7AD6EB30E04009EA8FDD72F
:10398000AD6EE20EF66E200EF76E410E0101BF6FB6
:10399000000193DDB30E04009EA8FDD7AD6E0D0EA1
:1039A00004009EA8FDD7AD6E0A0E04009EA8FDD7A8
:1039B000AD6E14DE000C0ADC010E0101BD6F250E98
:1039C000BE6F280EBF6F00016EDC640EF66E280E0F
:1039D000F76E98DCA9DCB00EF66E280EF76E92DC5E
:1039E000040EF66E260EF76E8DDC2E0E04009EA8D9
:1039F000FDD7AD6E200E04009EA8FDD7AD6E180E4B
:103A0000F66E260EF76E7EDCBC0EF66E280EF76E96
:103A100079DC260EF66E260EF76E74DC2E0E040090
:103A20009EA8FDD7AD6E0D0E04009EA8FDD7AD6E0D
:103A30000A0E04009EA8FDD7AD6EC40EF66E280EC9
:103A4000F76E60DC360EF66E260EF76E5BDC0D0E42
:103A500004009EA8FDD7AD6E0A0E04009EA8FDD7F7
:103A6000AD6E0A0E04009EA8FDD7AD6ED40EF66EA4
:103A7000280EF76E47DC010E0101BD6F250EBE6FEB
:103A8000280EBF6F00010FDC310E1B5CCE0FD8B0CB
:103A900078D0320F14EF1EF0A80EF66E240EF76EDB
:103AA00031DC6FD0BE0EF66E240EF76E2BDC69D0C3
:103AB000060EF66E250EF76E25DC63D0180EF66E38
:103AC000250EF76E1FDC5DD02E0EF66E250EF76EFE
:103AD00019DC57D03E0EF66E250EF76E13DC51D072
:103AE000520EF66E250EF76E0DDC4BD0620EF66EA2
:103AF000250EF76E07DC45D0760EF66E250EF76EB6
:103B000001DC3FD0800EF66E250EF76E82EC19F0C8
:103B100038D0900EF66E250EF76E82EC19F031D08B
:103B20009C0EF66E250EF76E82EC19F02AD0AC0EC4
:103B3000F66E250EF76E82EC19F023D0C20EF66EEB
:103B4000250EF76E82EC19F01CD0DA0EF66E250EFB
:103B5000F76E82EC19F015D0E80EF66E250EF76EB2
:103B600082EC19F00ED0D80EF66E240EF76E82ECB1
:103B700019F007D0F20EF66E240EF76E82EC19F0F3
:103B800000D0D89224C1D0F123C1CFF122C1CEF10F
:103B900021C1CDF10101D46B0F0ED36F420ED26F54
:103BA000400ED16F0001B4EC19F003C0C0F102C0A7
:103BB000BFF101C0BEF100C0BDF1200E04009EA8FF
:103BC000FDD7AD6E2D0E04009EA8FDD7AD6E200E64
:103BD00004009EA8FDD7AD6E410EE96EC0C1C4F1D0
:103BE000BFC1C3F1BEC1C2F1BDC1C1F107DC6D0EE1
:103BF00004009EA8FDD7AD6E6C0E04009EA8FDD7F4
:103C0000AD6E94EC19F00D0E04009EA8FDD7AD6EBC
:103C10000A0E04009EA8FDD7AD6E0A0E04009EA8F1
:103C2000FDD7AD6EFDDC000CE824F76AF736430FD4
:103C3000F66E3C0EF7220A00F550FA6E0800F550B9
:103C4000F96E983AA43AB03ABC3AC83AD43AE03A53
:103C5000EC3AF83A043B123B203B2E3B3C3B4A3BC0
:103C6000583B823B823B823B823B823B823B823B96
:103C7000823B823B823B823B823B823B823B823B5C
:103C8000823B823B823B823B823B823B823B823B4C
:103C9000823B823B823B823B823B823B823B823B3C
:103CA000823B663B743B010EEA6EC20EE96EEF503A
:103CB00011E0060E016EBF0E006E0400002EFDD74F
:103CC000012EF9D77A0E006E002EFED700D0040028
:103CD000EF2EEFD7000C93928A82010E0101C26F82
:103CE0000001E1DF000C93948A840400180E006E3A
:103CF000002EFED7000093968A860400180E006EF0
:103D0000002EFED7000093968A960400180E006ECF
:103D1000002EFED7000093948A940400100E006ECB
:103D2000002EFED70101BD6BBD511F081FE3939606
:103D30008A8604000B0E006E002EFED7938081B0A1
:103D400002D0D89001D0D880C133C033BF33BE3346
:103D500004000B0E006E002EFED793968A96040088
:103D6000290E006E002EFED7BD2BDED7010EC26FCE
:103D7000000199DFBEC100F0BFC101F0C0C102F077
:103D8000C1C103F0000C93800400180E006E002ED9
:103D9000FED7000093968A860400200E006E002E47
:103DA000FED700D093908A900400180E006E002E6B
:103DB000FED7000093968A960400180E006E002E1F
:103DC000FED70000000C93908A900400100E006E45
:103DD000002EFED793968A860400070E006E002EF2
:103DE000FED700D0938004000B0E006E002EFED78D
:103DF00093968A960400180E006E002EFED70000DF
:103E0000000CBDC1C1F1BEC1C2F1BFC1C3F1BBDF76
:103E10000101C06BC051170820E3D890C333C233EF
:103E2000C13302E3938002D093908A900400070E7E
:103E3000006E002EFED700D093968A860400100EE6
:103E4000006E002EFED793968A960400070E006E31
:103E5000002EFED700D0C02BDDD70001B4DF000C50
:103E60000101C06BBF5308E193968A960400200EAF
:103E7000006E002EFED700D0C16BC15107081CE3B5
:103E800093968A8604000B0E006E002EFED7938058
:103E900081B002D0D89001D0D880C03304000B0E7E
:103EA000006E002EFED793968A960400150E006EC3
:103EB000002EFED7C12BE1D7C0C101F00001000CDC
:103EC000010E0101C26F0001EEDE93928A92000C96
:103ED00092908990000CD190938881B82ED0FF0EDB
:103EE00001012C6F2B6F2A6F296F2551295D09E184
:103EF00026512A5D06E127512B5D03E128512C5DF7
:103F000014E0000158DD0101BC6BBB6BBC51000823
:103F10000CE31D0EBB25E96E000EBC21EA6EFF0E00
:103F2000EF6EBB2BD8B4BC2BF1D7FF0E286F276FD9
:103F3000266F256FD180E2D00001CDDED4DE300EB9
:103F40000101BD6FBE6BBF6B00015BDF0101BF6B89
:103F5000000186DF01C01DF0010E0101BF6F0001ED
:103F60007FDF01C01EF0010E0101BF6F000178DF8D
:103F700001C01FF0010E0101BF6F000171DF01C020
:103F800020F093948A840400A60E006E002EFED7C3
:103F900093948A9495DF1DC02CF11EC02BF11FC095
:103FA0002AF120C029F101012551295D14E1265192
:103FB0002A5D11E127512B5D0EE128512C5D0BE1AB
:103FC000000E1AB2010EBD6F9388000E81B8010E6B
:103FD000BD5DD8B492D000017EDE85DE79DF0101BF
:103FE000BC6B040EBB6FBC51000877E3300EBD6F95
:103FF000BBC1BEF1BF6B000104DF1D0E0101BB257B
:10400000016E000EBC21036E01C0BDF1BE6FBF6B1F
:10401000000126DFBEC1EAFFBDC1E9FF01C0EFFF1D
:10402000010E0101BB25BD6F000EBC21BE6F1D0E30
:10403000BD25016E000EBE21036E01C0BDF1BE6F35
:10404000010EBF6F00010CDFBEC1EAFFBDC1E9FF79
:1040500001C0EFFF020E0101BB25BD6F000EBC21A8
:10406000BE6F1D0EBD25016E000EBE21036E01C088
:10407000BDF1BE6F010EBF6F0001F2DEBEC1EAFFEF
:10408000BDC1E9FF01C0EFFF030E0101BB25BD6FFC
:10409000000EBC21BE6F1D0EBD25016E000EBE219F
:1040A000036E01C0BDF1BE6F010EBF6F0001D8DE0F
:1040B000BEC1EAFFBDC1E9FF01C0EFFF93948A844E
:1040C0000400A60E006E002EFED793948A94040E70
:1040D0000101BB27000EBC2386D70001F1DE6BDC9B
:1040E0002CC128F12BC127F12AC126F129C125F1C4
:1040F00093881A9281B81A820101D180F29400014A
:1041000030EF04F04F7074696F6E2073656C6563F7
:104110007465642E2E2E25430D0A0000456E7465CD
:104120007220612032206469676974206865782094
:1041300076616C756520746F2070726F6772616D47
:1041400020746F207468652063617264202D2000E4
:10415000456E74657220612032206469676974203D
:104160006865782064657374696E6174696F6E2028
:1041700061646472657373202D2000000D0A496E1E
:104180007075742038206368617261637465722091
:104190006865782050726F74656374696F6E207003
:1041A00061747465726E3A200000938093928A92D3
:1041B00093948A9493968A9600EF58F09280000C1C
:1041C00061C1AAFF60C1A9FF62C1A8FFA69CA69E0B
:1041D000A684F250006EF29E0F01550EA76EAA0E35
:1041E000A76EA682A6B2FED7A6940050F2120001D6
:1041F000000C1B0E04009EA8FDD7AD6E630E0400DC
:104200009EA8FDD7AD6E07EF5AF0196AF2BE198E5F
:10421000F29E020E0101BD6F250EBE6F280EBF6F0C
:10422000000153EC19F019BEF28E01014F6B4F5192
:1042300018080DE3506B50514F0807E3200E04009F
:104240009EA8FDD7AD6E502BF6D74F2BF0D7196A2D
:10425000F2BE198EF29E000194EC19F019BEF28E96
:1042600009EF5AF0EACF77F1E9CF76F10101703921
:10427000F009726F7227E20F736F320F756F705112
:104280000F0B732773277527E90F746F7427742733
:104290006F390F0B7427752774377537751F75378E
:1042A0006F510F0B75277237070E716F0A0E740767
:1042B0007527FDE373077427FDE372077327FDE39A
:1042C00071077227FDE3010EEA6E710EE96E070EAB
:1042D0007615769DE926750EE95CD8B4768DEF509B
:1042E000006E08E176BD06D076B90DD076B702D063
:1042F000200E03D076877699300E002600500400F9
:104300009EA8FDD7AD6EEE5076ADE5D70001000C4E
:10431000F2CF61F1F29EAA6A100EA96EA69CA69E2B
:10432000A680A850010161BFF28E626FF2CF63F1E7
:10433000F29EAA6A110EA96EA69CA69EA680A850FF
:1043400063BFF28E646F62C15CF164C15BF15C516A
:10435000260837E2FF0A03E15B51100832E25C6B8A
:10436000320E5B6F5CC161F1626BAA6A100EA96EBE
:1043700061C1A8FFA69CA69EA684F250006EF29E84
:104380000F01550EA76EAA0EA76EA682A6B2FED783
:10439000A6940050F212AA6A110EA96E5BC1A8FF82
:1043A000A69CA69EA684F2CF00F0F29E550EA76EA4
:1043B000AA0EA76EA682A6B2FED7A6940050F2124D
:1043C00001015B5323E15C5321E11A0EF66E2B0EC3
:1043D000F76E196AF2BE198EF29E000182EC19F096
:1043E00019BEF28E080E0101616F196AF2BE198EB4
:1043F000F29EFA0EC26F000156DC19BEF28E010168
:10440000612FF3D7000E016EB1D0B0D05C536AE1DA
:104410005B51310867E3520EF66E2B0EF76E196A88
:10442000F2BE198EF29E170EBF6F00015DEC1AF0FE
:1044300019BEF28E100EE96E5CC170F15BC16FF1B6
:1044400011DF6C0EF66E2B0EF76E196AF2BE198E26
:10445000F29E070E0101BF6F00015DEC1AF019BE5C
:10446000F28E01015C5303E15B51010805E2730E1A
:1044700004009EA8FDD7AD6E740EF66E2B0EF76E7F
:10448000196AF2BE198EF29E000182EC19F019BE73
:10449000F28E040EF66E260EF76E196AF2BE198EB3
:1044A000F29E82EC19F019BEF28E9A0EF66E2B0E69
:1044B000F76E196AF2BE198EF29E82EC19F019BEDF
:1044C000F28E080E0101616F196AF2BE198EF29E1A
:1044D000FA0EC26F000153EC1EF019BEF28E0101FC
:1044E000612FF2D7F2CF61F1F29EAA6A160EA96E81
:1044F000A69CA69EA680A85061BFF28E626FF2CFE6
:1045000063F1F29EAA6A170EA96EA69CA69EA680CB
:10451000A85063BFF28E646FF2CF65F1F29EAA6A73
:10452000180EA96EA69CA69EA680A85065BFF28E06
:10453000666F606B62C15FF164C15EF166C15DF17F
:104540005D51DD0810E15E5126080DE15F530BE17E
:10455000605309E15C5307E15B511D0804E3000E61
:10456000016E04D003D0010E016E00D00001000CDA
:1045700025DE640EF66E230EF76E196AF2BE198EF2
:10458000F29E82EC19F019BEF28E04009EAAFDD7AD
:10459000AE50000C01017A6B796B938081B014D01E
:1045A00093968A860400180E006E002EFED7000037
:1045B00093968A960400180E006E002EFED7000017
:1045C000792BD8B47A2BE9D779C101F07AC102F0FE
:1045D0000001000C01017ABF11D00F0E006E793975
:1045E00000160A0E005C03E2300E002602D07A515B
:1045F0000026005004009EA8FDD7AD6E0F0E79175F
:104600000A0E795D02E2300E02D07A9F7A51792744
:10461000795104009EA8FDD7AD6E0001000C196A07
:10462000F2BE198EF29E6BEC1EF019BEF28E196A64
:10463000F2BE198EF29E73EC1EF019BEF28E48DCAB
:10464000196AF2BE198EF29E340E0101BD6FBE6B67
:10465000BF6B000101EC1FF019BEF28E0101765311
:1046600014E0775304E00001E6EC18F001015E0E5F
:10467000F66E260EF76E196AF2BE198EF29E0001D2
:1046800082EC19F019BEF28E0101786B78510308A3
:104690001EE3036A78511D0F016E010E032201C053
:1046A00079F103C07AF1196AF2BE198EF29E78C1CF
:1046B000BFF1000130EC1FF019BEF28E7AC1EAFFA3
:1046C00079C1E9FF01C0EFFF0101782BDFD70001BD
:1046D00061DF196AF2BE198EF29E60EC1FF019BEFE
:1046E000F28E6CDD010176533AE020C179F1370E8C
:1046F0007A6F00016FDF200E04009EA8FDD7AD6E1B
:104700001FC179F1370E01017A6F000163DF200EBE
:1047100004009EA8FDD7AD6E1EC179F1370E0101D0
:104720007A6F000157DF200E04009EA8FDD7AD6E02
:104730001DC179F1370E01017A6F00014BDF0D0EBB
:1047400004009EA8FDD7AD6E0A0E04009EA8FDD7FA
:10475000AD6E0A0E04009EA8FDD7AD6E01010001EA
:10476000000CE6EC18F0C60EF66E260EF76E196A0F
:10477000F2BE198EF29E82EC19F019BEF28ED00EA6
:10478000F66E260EF76E196AF2BE198EF29E82EC54
:1047900019F019BEF28E200EF66E270EF76E196A0A
:1047A000F2BE198EF29E82EC19F019BEF28E720ED4
:1047B000F66E270EF76E196AF2BE198EF29E82EC23
:1047C00019F019BEF28E860EF66E270EF76E196A74
:1047D000F2BE198EF29E82EC19F019BEF28EC8DE7E
:1047E000000C01015F81766B010E776F000117DF0E
:1047F00020C15EF11FC15DF11EC15CF11DC15BF105
:1048000001015B51006E5C51036EFF0E035C05E11C
:10481000FF0E005C00010AE00101FF0E035C05E1F0
:10482000F00E005C000103E001014BD050D001010B
:104830002951006E2A51036E100E035C05E1910EA2
:10484000005C00010AE00101100E035C05E1880E26
:10485000005C000110E0010116D01B50300803E29B
:104860001B50320803E21B50610804E17ADF0101AA
:104870005F91000125D01B50020804E272DF0101A4
:104880005F9100011DD00001E6EC18F09C0EF66E61
:10489000270EF76E196AF2BE198EF29E82EC19F09D
:1048A00019BEF28EDC0EF66E270EF76E196AF2BE96
:1048B000198EF29E82EC19F019BEF28E59DE00D0EC
:1048C00006D000014EDF01015F91000100D0000E13
:1048D00001015FB1010E016E0001000C01015D518B
:1048E0005F03F3CF01F0F4CF00F06003F350002634
:1048F0005E515F03F3500020026E0001000C0101C5
:104900005B531FE1D892196AF2BE198EF29E24C140
:10491000D0F123C1CFF122C1CEF121C1CDF1D46BB1
:104920000F0ED36F420ED26F400ED16F0001B4EC68
:1049300019F019BEF28E01C05FF100C05EF105D022
:1049400001015DC15FF15CC15EF101015F5312E1E4
:104950005E51DC080FE35B5303E1FF0E386E09D0B4
:10496000010E616F1B0E606FFF0E626F000128DC8D
:1049700001016BD05F51030813E303E15E51E708C7
:104980000FE35B5303E1010E386E09D0010E616F36
:104990001B0E606F010E626F000112DC010155D029
:1049A0005F51070814E303E15E51CF0810E35B5346
:1049B00003E1020E386E0AD0010E616F1B0E606FAC
:1049C000020E626F0001E0EC20F001013ED05F5169
:1049D0000B0814E303E15E51B70810E35B5303E1F6
:1049E000030E386E0AD0010E616F1B0E606F030E4E
:1049F000626F0001E0EC20F0010127D05F510F0849
:104A000015E303E15E519F0811E35B5303E1040EDC
:104A1000386E0AD0010E616F1B0E606F040E626F5C
:104A20000001E0EC20F0010110D00FD05B5303E156
:104A3000050E386E0AD0010E616F1B0E606F050EF9
:104A4000626F0001E0EC20F001010001000C1B0E80
:104A500004009EA8FDD7AD6E5B0E04009EA8FDD796
:104A6000AD6E730E04009EA8FDD7AD6E000C196AE2
:104A7000F2BE198EF29E310E0101BD6FBE6BBF6B8F
:104A8000000101EC1FF019BEF28E0101606B605154
:104A900003081EE3036A60515C0F016E010E0322DE
:104AA00001C064F103C065F1196AF2BE198EF29E6D
:104AB00060C1BFF1000130EC1FF019BEF28E65C17C
:104AC000EAFF64C1E9FF01C0EFFF0101602BDFD7FE
:104AD0005B534AE00001E6EC18F0820EF66E260EFB
:104AE000F76E196AF2BE198EF29E82EC19F019BEA9
:104AF000F28E5FC179F1370E01017A6F00016ADD34
:104B0000200E04009EA8FDD7AD6E5EC179F1370E70
:104B100001017A6F00015EDD200E04009EA8FDD722
:104B2000AD6E5DC179F1370E01017A6F000152DD82
:104B3000200E04009EA8FDD7AD6E5CC179F1370E42
:104B400001017A6F000146DD0D0E04009EA8FDD71D
:104B5000AD6E0A0E04009EA8FDD7AD6E0A0E0400CD
:104B60009EA8FDD7AD6E01015C51070B616F6151CD
:104B7000F80FD8B0FDD1080F000127EF2AF001018E
:104B80005B531AE0BA0EF66E210EF76E196AF2BE8A
:104B9000198EF29E000182EC19F019BEF28EF00E11
:104BA000F66E210EF76E196AF2BE198EF29E82EC35
:104BB00019F019BEF28E0101040E646F196AF2BE7B
:104BC000198EF29EFA0EC26F000153EC1EF019BE50
:104BD000F28E0101642FF2D7000E016E24EF2AF04D
:104BE000000101015B532EE0700EF66E210EF76E90
:104BF000196AF2BE198EF29E2B0EBF6F00015DEC9A
:104C00001AF019BEF28E196AF2BE198EF29E020EC9
:104C10000101C06F1B0EC16F000111EC19F019BE2C
:104C2000F28E9D0EF66E210EF76E196AF2BE198E87
:104C3000F29E1B0E0101BF6F00015DEC1AF019BE60
:104C4000F28E0101196AF2BE198EF29E390EBD6F05
:104C5000BE6BFE0EBF6F000101EC1FF019BEF28E9D
:104C6000010186D101015B532EE0700EF66E210E1C
:104C7000F76E196AF2BE198EF29E2B0EBF6F0001FD
:104C80005DEC1AF019BEF28E196AF2BE198EF29E10
:104C9000020E0101C06F1B0EC16F000111EC19F073
:104CA00019BEF28E9D0EF66E210EF76E196AF2BED7
:104CB000198EF29E1B0E0101BF6F00015DEC1AF010
:104CC00019BEF28E0101196AF2BE198EF29E390EDA
:104CD000BD6FBE6BFE0EBF6F000101EC1FF019BE71
:104CE000F28E010145D101015B532EE0700EF66E8C
:104CF000210EF76E196AF2BE198EF29E2B0EBF6F4F
:104D000000015DEC1AF019BEF28E196AF2BE198E1E
:104D1000F29E020E0101C06F1B0EC16F000111EC6B
:104D200019F019BEF28E9D0EF66E210EF76E196AFD
:104D3000F2BE198EF29E1B0E0101BF6F00015DECE9
:104D40001AF019BEF28E0101196AF2BE198EF29E96
:104D5000390EBD6FBE6BFD0EBF6F000101EC1FF081
:104D600019BEF28E010104D101015B532EE0700ED9
:104D7000F66E210EF76E196AF2BE198EF29E2B0E98
:104D8000BF6F00015DEC1AF019BEF28E196AF2BE17
:104D9000198EF29E010E0101C06F1B0EC16F000142
:104DA00011EC19F019BEF28E9D0EF66E210EF76E03
:104DB000196AF2BE198EF29E1B0E0101BF6F00012F
:104DC0005DEC1AF019BEF28E0101196AF2BE198E5D
:104DD000F29E390EBD6FBE6BFE0EBF6F000101EC7F
:104DE0001FF019BEF28E0101C3D001015B532EE00A
:104DF000700EF66E210EF76E196AF2BE198EF29ED3
:104E00002B0EBF6F00015DEC1AF019BEF28E196A0D
:104E1000F2BE198EF29E010E0101C06F1B0EC16F12
:104E2000000111EC19F019BEF28E9D0EF66E210EE6
:104E3000F76E196AF2BE198EF29E1B0E0101BF6F4A
:104E400000015DEC1AF019BEF28E0101196AF2BE82
:104E5000198EF29E390EBD6FBE6BFD0EBF6F000145
:104E600001EC1FF019BEF28E010182D001015B53EB
:104E70002EE0700EF66E210EF76E196AF2BE198ED4
:104E8000F29E2B0EBF6F00015DEC1AF019BEF28E80
:104E9000196AF2BE198EF29E010E0101C06F1B0E3F
:104EA000C16F000111EC19F019BEF28E9D0EF66E65
:104EB000210EF76E196AF2BE198EF29E1B0E0101C9
:104EC000BF6F00015DEC1AF019BEF28E0101196A84
:104ED000F2BE198EF29E390EBD6FBE6BFB0EBF6F18
:104EE000000101EC1FF019BEF28E010141D0010159
:104EF0005B532EE0700EF66E210EF76E196AF2BE4D
:104F0000198EF29E2B0EBF6F00015DEC1AF019BED8
:104F1000F28E196AF2BE198EF29E030E0101C06F65
:104F20001B0EC16F000111EC19F019BEF28E9D0E1F
:104F3000F66E210EF76E196AF2BE198EF29E1B0EE6
:104F40000101BF6F00015DEC1AF019BEF28E010184
:104F5000196AF2BE198EF29E390EBD6FBE6BFE0E3F
:104F6000BF6F000101EC1FF019BEF28E010100D0ED
:104F70000001CAEC22F001C063F101015B530FE0B4
:104F80000D0E04009EA8FDD7AD6E0A0E04009EA86B
:104F9000FDD7AD6E0A0E04009EA8FDD7AD6E196A4E
:104FA000F2BE198EF29E330EBD6F010EBE6FFF0E64
:104FB000BF6F000101EC1FF019BEF28ECAEC22F0A7
:104FC000196AF2BE198EF29E330E0101BD6F020EF8
:104FD000BE6FFF0EBF6F000101EC1FF019BEF28E15
:104FE000CAEC22F0196AF2BE198EF29E330E01014C
:104FF000BD6F030EBE6FFF0EBF6F000101EC1FF00F
:1050000019BEF28ECAEC22F0196AF2BE198EF29E17
:10501000390E0101BD6FBE6BFF0EBF6F000101ECC9
:105020001FF019BEF28ECAEC22F001C063F1196ABA
:10503000F2BE198EF29E310E0101BD6FBE6BBF6BC9
:10504000000101EC1FF019BEF28E0101606B60518E
:1050500003081EE3036A60515C0F016E010E032218
:1050600001C064F103C065F1196AF2BE198EF29EA7
:1050700060C1BFF1000130EC1FF019BEF28E65C1B6
:10508000EAFF64C1E9FF01C0EFFF0101602BDFD738
:105090005B534CE0A40EF66E260EF76E196AF2BE54
:1050A000198EF29E000182EC19F019BEF28E5FC1DA
:1050B00079F1370E01017A6F0001EAEC22F0200E3F
:1050C00004009EA8FDD7AD6E5EC179F1370E0101D7
:1050D0007A6F0001EAEC22F0200E04009EA8FDD7B2
:1050E000AD6E5DC179F1370E01017A6F0001EAEC16
:1050F00022F0200E04009EA8FDD7AD6E5CC179F1B0
:10510000370E01017A6F0001EAEC22F00D0E040067
:105110009EA8FDD7AD6E0A0E04009EA8FDD7AD6E09
:105120000A0E04009EA8FDD7AD6E01015B53D8B4F2
:1051300089D15C51070B626F6251F80FD8B082D1F0
:10514000080F00013CEF2AF0BA0EF66E210EF76E42
:10515000196AF2BE198EF29E82EC19F019BEF28E17
:10516000F00EF66E210EF76E196AF2BE198EF29EDF
:1051700082EC19F019BEF28E040E0101646F196AF7
:10518000F2BE198EF29EFA0EC26F000153EC1EF0B1
:1051900019BEF28E0101642FF2D7000E016E54D1B8
:1051A0000001700EF66E210EF76E196AF2BE198EAE
:1051B000F29E2B0E0101BF6F00015DEC1AF019BECB
:1051C000F28E196AF2BE198EF29E020E0101C06FB4
:1051D0001B0EC16F000111EC19F019BEF28E9D0E6D
:1051E000F66E210EF76E196AF2BE198EF29E1B0E34
:1051F0000101BF6F00015DEC1AF019BEF28E0101D2
:1052000021D1700EF66E210EF76E196AF2BE198E5C
:10521000F29E2B0E0101BF6F00015DEC1AF019BE6A
:10522000F28E196AF2BE198EF29E020E0101C06F53
:105230001B0EC16F000111EC19F019BEF28E9D0E0C
:10524000F66E210EF76E196AF2BE198EF29E1B0ED3
:105250000101BF6F00015DEC1AF019BEF28E010171
:10526000F1D0700EF66E210EF76E196AF2BE198E2D
:10527000F29E2B0E0101BF6F00015DEC1AF019BE0A
:10528000F28E196AF2BE198EF29E020E0101C06FF3
:105290001B0EC16F000111EC19F019BEF28E9D0EAC
:1052A000F66E210EF76E196AF2BE198EF29E1B0E73
:1052B0000101BF6F00015DEC1AF019BEF28E010111
:1052C000C1D0700EF66E210EF76E196AF2BE198EFD
:1052D000F29E2B0E0101BF6F00015DEC1AF019BEAA
:1052E000F28E196AF2BE198EF29E010E0101C06F94
:1052F0001B0EC16F000111EC19F019BEF28E9D0E4C
:10530000F66E210EF76E196AF2BE198EF29E1B0E12
:105310000101BF6F00015DEC1AF019BEF28E0101B0
:1053200091D0700EF66E210EF76E196AF2BE198ECC
:10533000F29E2B0E0101BF6F00015DEC1AF019BE49
:10534000F28E196AF2BE198EF29E010E0101C06F33
:105350001B0EC16F000111EC19F019BEF28E9D0EEB
:10536000F66E210EF76E196AF2BE198EF29E1B0EB2
:105370000101BF6F00015DEC1AF019BEF28E010150
:1053800061D0700EF66E210EF76E196AF2BE198E9C
:10539000F29E2B0E0101BF6F00015DEC1AF019BEE9
:1053A000F28E196AF2BE198EF29E010E0101C06FD3
:1053B0001B0EC16F000111EC19F019BEF28E9D0E8B
:1053C000F66E210EF76E196AF2BE198EF29E1B0E52
:1053D0000101BF6F00015DEC1AF019BEF28E0101F0
:1053E00031D0700EF66E210EF76E196AF2BE198E6C
:1053F000F29E2B0E0101BF6F00015DEC1AF019BE89
:10540000F28E196AF2BE198EF29E030E0101C06F70
:105410001B0EC16F000111EC19F019BEF28E9D0E2A
:10542000F66E210EF76E196AF2BE198EF29E1B0EF1
:105430000101BF6F00015DEC1AF019BEF28E01018F
:1054400001D00101010E016E000168EF2AF0E8248D
:10545000F76AF736690FF66E540EF7220A00F55018
:10546000FA6E0800F550F96E7E4B684DEA4DE24B3E
:105470006C4E644CE64CEE4EE824F76AF736930F18
:10548000F66E540EF7220A00F550FA6E0800F55039
:10549000F96E4851C2522253A251825302526252B3
:1054A000E25368EC1FF0196AF2BE198EF29E6BECA3
:1054B0001EF019BEF28E196AF2BE198EF29E73ECBE
:1054C0001EF019BEF28E01015B6B000137EF25F073
:1054D000000C1B0E04009EA8FDD7AD6E5B0E0400F1
:1054E0009EA8FDD7AD6E750E04009EA8FDD7AD6ECB
:1054F000000C196AF2BE198EF29E010E0101BD6FF9
:10550000250EBE6F280EBF6F000153EC19F019BEB7
:10551000F28E240EF66E280EF76E196AF2BE198E00
:10552000F29E82EC19F019BEF28E196AF2BE198E43
:10553000F29E94EC19F019BEF28E000CB60E006EBD
:10554000036A026A016A01017651771178117911B3
:1055500002E1006A0DD0D89001BE09D076377737C6
:1055600078377937033602360136002EF4D7019E9C
:105570000001000CE95001017E6F7DAF0DD07E0768
:105580007E8B7A1F7B1F7C1F7D1F7A2BD8B47B2BD1
:10559000D8B47C2BD8B47D2B3B0E856F9A0E846FCC
:1055A000CA0E836F826B0A0E806FD882010EEA6E7C
:1055B0007A0EE96E196AF2BE198EF29E7DC1D0F1A3
:1055C0007CC1CFF17BC1CEF17AC1CDF185C1D4F1DF
:1055D00084C1D3F183C1D2F182C1D1F10001B4EC15
:1055E00019F019BEF28E0150005213E101018051F1
:1055F000010AD8A402D000010CD07E510DE00F0B9F
:10560000805D01E02BE27EBF29D07EBD05D0200E5B
:105610001FD0200E01017E177EAB0BD07E9B00C0F9
:105620007EF12D0E04009EA8FDD7AD6E7EC100F068
:105630007E6B300E7EAB0CD07E9B00C07EF12D0EBB
:1056400004009EA8FDD7AD6E7EC100F07E6B300ECB
:105650000026005004009EA8FDD7AD6ED892196AAE
:10566000F2BE198EF29E85C1D0F184C1CFF183C103
:10567000CEF182C1CDF1D46BD36BD26B0A0ED16F58
:105680000001B4EC19F019BEF28E03C085F102C01E
:1056900084F101C083F100C082F10101802F85D720
:1056A0000001CFEF30F0800ED8A202D001017B1BA9
:1056B0000101806B816B77C17FF17B517F1B76513C
:1056C000D8B4DFD07E6F006E7A51D8B4E3D07E5F5D
:1056D000D8B483D03EE37BC184F1848F7CC183F155
:1056E0007DC182F1816BD8908433833382338133DF
:1056F0007E2FF8D77FAF03D08081E0D080917E915C
:105700008089010EEA6E790EE96EEBD080997FBF39
:105710000AD07EA113D08433833382338133002AAD
:10572000D8B4C7D00BD084BF0CD0D8908137823783
:10573000833784370006D8B4BCD0F5D7808D6DD0C0
:10574000809D77C17FF177AF02D0848FABD0849FEB
:10575000A9D07AC17EF17AC100F076517E5F77C11F
:1057600084F1848F78C183F179C182F1816BD89003
:1057700084338333823381337E2FF8D77FAF03D0D6
:1057800080839CD080937E91808B010EEA6E7D0E8B
:10579000E96EA7D0809B7FBF0AD07EA113D084334F
:1057A000833382338133002AD8B483D00BD084BFB3
:1057B0000CD0D89081378237833784370006D8B42D
:1057C00078D0F5D7808F29D0809F7BC17FF17BAFC8
:1057D00002D0848F67D0849F65D07BC184F1848F91
:1057E0007CC183F17DC182F17FAF04D0849F80852D
:1057F00065D08095816B7E91010EEA6E790EE96E1F
:1058000070D07FBF1CD077C17FF17EA106D08433DA
:10581000833382338133002A4CE081AF0BD0822B5B
:1058200009E1832B07E1842B05E184338333823341
:10583000002A3FE080BD84D780BFC6D71CD0800E31
:10584000841B84AF04D03AD07BC17FF10AD077C1EA
:105850007FF1845306E1835304E1825302E1006A3D
:1058600021D084BF08D0D8908137823783378437DE
:10587000002EF7D71ED07FAF02D0848F13D0849F25
:1058800011D07AC100F07BC184F17CC183F17DC16C
:1058900082F108D076C100F077C184F178C183F13C
:1058A00079C182F184C101F083C102F082C103F0A9
:1058B00034D0006A016A026A036A2FD0816B821FAA
:1058C000831F841F811F812B05E1822B03E1832B22
:1058D00001E1842B80B112D780B354D780B589D72A
:1058E000B3D7EF50822705E3832B03E1842BD8B491
:1058F0007E81ED52EF50832703E3842BD8B47E8161
:10590000ED52EF50EFBE01D0800A8427D8B07E81DF
:1059100080B9FCD680BB3ED774D700012FEF31F0A1
:1059200001017A51D8B4A5D0866F7E51D8B4A1D0E8
:10593000865F05E37F0E8627D8B09BD006D0810E08
:10594000865FD8A096D0D8B494D086C100F0016A02
:10595000026A036A856B7BC184F1848F7CC183F109
:105960007DC182F1190E866F8151825F0DE2010EB9
:10597000835F0AE2845F08E2855F06E2852B842B61
:10598000832B8151822728D08051835F12E2010E40
:10599000845F0FE2855F0DE2852B842B8051832786
:1059A0008151822719E3832B17E1842B15E1852B85
:1059B00013D07F518009845F0EE2010E855F0BE2F8
:1059C000852B7F518009842780518327E9E3842B2D
:1059D000E7E1852BE5D70380862F01D00BD0D89047
:1059E0008237833784378537D890033602360136BD
:1059F0008737BAD787A106D0D89001320232033256
:105A0000873302D0000635E087BF1ED0D89082379A
:105A10008337843785378151825F07E2010E835FC8
:105A200004E2845F02E2855F1AE38051835F05E24E
:105A3000010E845F02E2855F12E37F518009845F7B
:105A400003E2010E855F0BE3032A09E1022A07E165
:105A5000012A05E1002A0DE00132023203327BC146
:105A600086F17F51861B86AF02D0018E06D0019E43
:105A700004D0006A016A026A036A00014AEF31F049
:105A800001018751D8B471D0006E8B51D8B46DD05C
:105A9000002604E3810E002668E204D07F0E005E3B
:105AA00064E363E088C18FF18C518F1B888F8C8FEA
:105AB0008A518E03F4CF91F189518D03F4CF03F015
:105AC000F3CF90F18E03F3509127F4509023000E02
:105AD00003228A518D03F3509127F4509023000E36
:105AE000026A0322022288518E03F3509027F45059
:105AF0000322000E022288518D03F3500326F45036
:105B00000222000E016A01228A518C03F350902771
:105B1000F4500322000E0222012289518C03F3501B
:105B20000326F4500222000E012288518C03F35008
:105B30000226F4500122002A01BE05D09037033618
:105B4000023601360006000E90AF0AD0032A022268
:105B50000122015005E1025003E1035001E1002A56
:105B60008FBF018E8FAF019E04D0006A016A026A66
:105B7000036A0001F4EF2DF001018751B608876F29
:105B8000036A88C18BF1888FD890883389338A3330
:105B90000332023201320032872FF6D78BAF0BD09F
:105BA000001E011E021E031E002AD8B4012AD8B40A
:105BB000022AD8B4032A000109EF2EF0E9500101AE
:105BC0007F6F7E51816F1BE07DC18AF17CC189F1BD
:105BD0007BC188F17AC187F18E6B8D6B200E8C6F43
:105BE000820E8B6F00014CD703C07DF102C07CF1A7
:105BF00001C07BF100C07AF10101812FE5D77DC1A1
:105C00008AF17CC189F17BC188F17AC187F10001F9
:105C1000B3D703C07DF102C07CF101C07BF100C0AD
:105C20007AF101017DAF0DD07F077F8B7A1F7B1F3B
:105C30007C1F7D1F7A2BD8B47B2BD8B47C2BD8B497
:105C40007D2B3B0E866F9A0E856FCA0E846F836B19
:105C50000A0E816F7E51D8B47F2BD882010EEA6E76
:105C60007A0EE96E196AF2BE198EF29E7DC1D0F1EC
:105C70007CC1CFF17BC1CEF17AC1CDF186C1D4F127
:105C800085C1D3F184C1D2F183C1D1F10001B4EC5B
:105C900019F019BEF28E0150005213E101017E2964
:105CA000815DD8A402D000010CD07F510DE00F0B14
:105CB000815D01E040E27FBF3ED07FBD05D0200E78
:105CC00034D0200E01017F177FAB0ED07F9B7E5119
:105CD000D8A47F0700507F6F2D0E04009EA8FDD72B
:105CE000AD6E7F51006E7F6B7E51815D0CE1005087
:105CF0007F6F2E0E04009EA8FDD7AD6E7F51006E03
:105D0000200E7F17000E300E7FAB0FD07F9B7E5191
:105D1000D8A47F0700507F6F2D0E04009EA8FDD7EA
:105D2000AD6E7F51006E7F6B300E00260050040078
:105D30009EA8FDD7AD6ED892196AF2BE198EF29E5A
:105D400086C1D0F185C1CFF184C1CEF183C1CDF13F
:105D5000D46BD36BD26B0A0ED16F0001B4EC19F087
:105D600019BEF28E03C086F102C085F101C084F134
:105D700000C083F10101812F70D7000161EF31F084
:105D8000E6EC18F001015B53D8A4A8EF33F0196AD0
:105D9000F2BE198EF29E010EBD6F250EBE6F280E4B
:105DA000BF6F000153EC19F019BEF28EC60EF66EED
:105DB0002B0EF76E196AF2BE198EF29E82EC19F064
:105DC00019BEF28E196AF2BE198EF29E94EC19F089
:105DD00019BEF28E79EC2AF001015F6B5E6B5F51A8
:105DE000000855E35E510F0B766F776B765336E103
:105DF000775334E1196AF2BE198EF29E010EBD6F1F
:105E0000250EBE6F280EBF6F000153EC19F019BEAE
:105E1000F28E0D0E04009EA8FDD7AD6E0A0E040092
:105E20009EA8FDD7AD6E5EC179F1370E01017A6F84
:105E30000001EAEC22F03A0E04009EA8FDD7AD6EF8
:105E4000200E04009EA8FDD7AD6E196AF2BE198E11
:105E5000F29E94EC19F019BEF28E01011D0E5E2522
:105E6000E96E000E5F21EA6EEFCF76F176C179F12F
:105E7000370E7A6F0001EAEC22F0200E04009EA893
:105E8000FDD7AD6E01015E2BD8B45F2BA8D75C5354
:105E9000D8B47CEF33F0F80EF66E2B0EF76E196A5D
:105EA000F2BE198EF29E000182EC19F019BEF28E3C
:105EB0004250010A13E0030A2EE0010A49E0070AF2
:105EC00064E0010AD8B47ED0030AD8B498D0F80AA6
:105ED000D8B4B2D0010AD8B4CCD0E8D0196AF2BE96
:105EE000198EF29E010E0101BD6F250EBE6F280EA8
:105EF000BF6F000153EC19F019BEF28E280EF66E3A
:105F0000240EF76E196AF2BE198EF29E82EC19F019
:105F100019BEF28ED8D0196AF2BE198EF29E010E09
:105F20000101BD6F240EBE6F280EBF6F000153EC40
:105F300019F019BEF28E380EF66E240EF76E196A3D
:105F4000F2BE198EF29E82EC19F019BEF28EBBD011
:105F5000196AF2BE198EF29E010E0101BD6F230E69
:105F6000BE6F280EBF6F000153EC19F019BEF28E00
:105F7000480EF66E240EF76E196AF2BE198EF29E66
:105F800082EC19F019BEF28E9ED0196AF2BE198EFB
:105F9000F29E010E0101BD6F210EBE6F280EBF6F74
:105FA000000153EC19F019BEF28E580EF66E240E55
:105FB000F76E196AF2BE198EF29E82EC19F019BEC4
:105FC000F28E81D0196AF2BE198EF29E020E010184
:105FD000BD6F240EBE6F280EBF6F000153EC19F089
:105FE00019BEF28E680EF66E240EF76E196AF2BEB6
:105FF000198EF29E82EC19F019BEF28E64D0196AE5
:10600000F2BE198EF29E020E0101BD6F230EBE6F0D
:10601000280EBF6F000153EC19F019BEF28E780EF6
:10602000F66E240EF76E196AF2BE198EF29E82EC9D
:1060300019F019BEF28E47D0196AF2BE198EF29E7F
:10604000020E0101BD6F1E0EBE6F2F0EBF6F00014D
:1060500053EC19F019BEF28E880EF66E240EF76E10
:10606000196AF2BE198EF29E82EC19F019BEF28EF8
:106070002AD0196AF2BE198EF29E020E0101BD6F7E
:106080001E0EBE6F2F0EBF6F000153EC19F019BE2C
:10609000F28E880EF66E240EF76E196AF2BE198E15
:1060A000F29E82EC19F019BEF28E0DD0980EF66EAB
:1060B000240EF76E196AF2BE198EF29E82EC19F068
:1060C00019BEF28E00D0196AF2BE198EF29E94ECBF
:1060D00019F019BEF28E45C065F146C064F147C0A3
:1060E00063F148C062F165C179F164C178F163C1BF
:1060F00077F162C176F19EEC2AF003C071F102C023
:1061000070F101C06FF100C06EF10A0EF66E2C0E38
:10611000F76E196AF2BE198EF29E82EC19F019BE62
:10612000F28E196AF2BE198EF29E010E0101BD6F48
:10613000250EBE6F280EBF6F000153EC19F019BE7B
:10614000F28ED892196AF2BE198EF29E65C1D0F114
:1061500064C1CFF163C1CEF162C1CDF10101D46B55
:106160000F0ED36F420ED26F400ED16F0001B4EC10
:1061700019F019BEF28E03C079F102C078F101C0A6
:1061800077F100C076F1040EE96E03C07DF102C024
:106190007CF101C07BF100C07AF1BAEF2AF06D0EFC
:1061A00004009EA8FDD7AD6E6C0E04009EA8FDD71E
:1061B000AD6E200E04009EA8FDD7AD6E196AF2BE2A
:1061C000198EF29E94EC19F019BEF28E49C069F155
:1061D0004AC068F14BC067F14CC066F169C179F102
:1061E00068C178F167C177F166C176F19EEC2AF05B
:1061F00003C075F102C074F101C073F100C072F107
:106200001C0EF66E2C0EF76E196AF2BE198EF29EF7
:1062100082EC19F019BEF28E196AF2BE198EF29E46
:10622000010E0101BD6F250EBE6F280EBF6F00016C
:1062300053EC19F019BEF28ED88271C179F170C198
:1062400078F16FC177F16EC176F175C17DF174C1DE
:106250007CF173C17BF172C17AF153EF2BF000C076
:1062600076F101C077F102C078F103C079F103C083
:106270007DF102C07CF101C07BF100C07AF1010127
:10628000816B240E806F740E7F6F920E7E6F000103
:1062900090EF2CF000C076F101C077F102C078F1E8
:1062A00003C079F1450EE96E03C07DF102C07CF1B7
:1062B00001C07BF100C07AF1030E01017E6F000185
:1062C0007DD46D0E04009EA8FDD7AD6E6C0E04004B
:1062D0009EA8FDD7AD6E196AF2BE198EF29E94EC9F
:1062E00019F019BEF28E3E0EF66E2C0EF76E196A7C
:1062F000F2BE198EF29E82EC19F019BEF28E41C0E8
:106300005FF144C05EF1196AF2BE198EF29E010E71
:106310000101BD6F250EBE6F280EBF6F000153EC4B
:1063200019F019BEF28E01015E51006E5F51036ECD
:10633000010E035C05E1080E005C000151E0010163
:10634000010E035C05E10D0E005C000156E0010149
:10635000010E035C05E1110E005C00015BE0010130
:10636000010E035C06E1130E005C0001D8B48CD072
:106370000101160E035C06E1110E005C0001D8B4A9
:1063800090D00101020E035C06E1070E005C0001E3
:10639000D8B494D00101080E035C06E1110E005C34
:1063A0000001D8B498D00101080E035C06E10D0E7F
:1063B000005C0001D8B49CD001010D0E035C06E125
:1063C0000D0E005C0001D8B4A0D00101090E035CE1
:1063D00006E1110E005C0001D8B4A4D00101B0D0D8
:1063E0004A0EF66E2C0EF76E196AF2BE198EF29EE8
:1063F00082EC19F019BEF28ED3D0640EF66E2C0E1C
:10640000F76E196AF2BE198EF29E82EC19F019BE6F
:10641000F28EC6D0293C01D02AD00101655318E183
:10642000645316E16351010813E303E16251B808B4
:106430000FE37E0EF66E2C0EF76E196AF2BE198E01
:10644000F29E000182EC19F019BEF28E0ED001010D
:10645000980EF66E2C0EF76E196AF2BE198EF29E29
:10646000000182EC19F019BEF28E9AD00DD0B20E56
:10647000F66E2C0EF76E196AF2BE198EF29E82EC41
:1064800019F019BEF28E8CD0CC0EF66E2C0EF76E73
:10649000196AF2BE198EF29E82EC19F019BEF28EC4
:1064A0007FD0E60EF66E2C0EF76E196AF2BE198ECC
:1064B000F29E82EC19F019BEF28E72D0000EF66ECA
:1064C0002D0EF76E196AF2BE198EF29E82EC19F04B
:1064D00019BEF28E65D01A0EF66E2D0EF76E196A81
:1064E000F2BE198EF29E82EC19F019BEF28E58D0CF
:1064F000340EF66E2D0EF76E196AF2BE198EF29EEC
:1065000082EC19F019BEF28E4BD04E0EF66E2D0EA7
:10651000F76E196AF2BE198EF29E82EC19F019BE5E
:10652000F28E3ED0680EF66E2D0EF76E196AF2BE30
:10653000198EF29E82EC19F019BEF28E31D0010153
:10654000820EF66E2D0EF76E196AF2BE198EF29E4D
:106550000A0EBF6F00015DEC1AF019BEF28E5FC12A
:1065600079F1370E01017A6F0001EAEC22F05EC189
:1065700079F1370E01017A6F0001EAEC22F08F0EFB
:10658000F66E2D0EF76E196AF2BE198EF29E0C0E83
:106590000101BF6F00015DEC1AF019BEF28E00D050
:1065A000196AF2BE198EF29E94EC19F019BEF28EA1
:1065B0000101766B776B00010FEC23F09C0EF66EF9
:1065C0002D0EF76E196AF2BE198EF29E82EC19F04A
:1065D00019BEF28E20C16DF11FC16CF11EC16BF1AD
:1065E0001DC16AF1196AF2BE198EF29E010E0101F7
:1065F000BD6F250EBE6F280EBF6F000153EC19F062
:1066000019BEF28E01016D51FF0839E30BE16C51A7
:10661000FF0835E307E16B51FF0831E303E16A51FD
:10662000EF082DE3B20EF66E2D0EF76E196AF2BE6C
:10663000198EF29E000182EC19F019BEF28E010152
:10664000616B606B61530CE16051350809E3200E0A
:1066500004009EA8FDD7AD6E602BD8B4612BF2D795
:10666000CC0EF66E2D0EF76E196AF2BE198EF29EE2
:10667000000182EC19F019BEF28E2CD00101E60E59
:10668000F66E2D0EF76E196AF2BE198EF29E00019B
:1066900082EC19F019BEF28E0101616B606B6153DF
:1066A0000CE16051350809E3200E04009EA8FDD7D7
:1066B000AD6E602BD8B4612BF2D7040EF66E2E0EA1
:1066C000F76E196AF2BE198EF29E000182EC19F083
:1066D00019BEF28E196AF2BE198EF29E94EC19F070
:1066E00019BEF28E0D0E04009EA8FDD7AD6E0A0EE7
:1066F00004009EA8FDD7AD6E0001DEEC20F0010184
:106700005D5325E00D0E04009EA8FDD7AD6E0A0E68
:1067100004009EA8FDD7AD6E0A0E04009EA8FDD70A
:10672000AD6E640EF66E230EF76E196AF2BE198E08
:10673000F29E000182EC19F019BEF28E9EBA06D0CC
:106740000400938881B801D001D0F8D70101A0D00E
:10675000196AF2BE198EF29E010EBD6F250EBE6F34
:10676000280EBF6F000153EC19F019BEF28E200EF7
:10677000F66E2E0EF76E196AF2BE198EF29E82EC3C
:1067800019F019BEF28E196AF2BE198EF29E94ECBF
:1067900019F019BEF28E79EC2AF001015F6B5E6B85
:1067A0005F51000860E35E510F0B766F776B765395
:1067B00036E1775334E1196AF2BE198EF29E010E6A
:1067C000BD6F250EBE6F280EBF6F000153EC19F090
:1067D00019BEF28E0D0E04009EA8FDD7AD6E0A0EF6
:1067E00004009EA8FDD7AD6E5EC179F1370E0101A0
:1067F0007A6F0001EAEC22F03A0E04009EA8FDD761
:10680000AD6E200E04009EA8FDD7AD6E196AF2BED3
:10681000198EF29E94EC19F019BEF28E01015E51B0
:10682000766F010E5F25776FF2CF78F1F29E77C118
:10683000AAFF76C1A9FFA69CA69EA680A85078BFF5
:10684000F28E766F76C179F1370E7A6F0001EAEC3D
:1068500022F0200E04009EA8FDD7AD6E01015E2B34
:10686000D8B45F2B9DD70D0E04009EA8FDD7AD6E4A
:106870000A0E04009EA8FDD7AD6E0A0E04009EA865
:10688000FDD7AD6E5D5304E00001B8EC22F00101CC
:106890000001000CEA0EF66E280EF76E196AF2BEC1
:1068A000198EF29E82EC19F019BEF28E04009EAA97
:1068B000FDD7AECF5BF101015B51600806E25B5191
:1068C0007A0803E35B51DF0B01D05B515B6F5B51D7
:1068D000590806E05B514E08D8B402D00001DAD75F
:1068E0005BC101F00001000C01015F6B5E6B5D5349
:1068F00004E00001E6EC18F00101F2CF60F1F29E35
:10690000AA6A100EA96EA69CA69EA680A85060BF7B
:10691000F28E616FF2CF62F1F29EAA6A110EA96E39
:10692000A69CA69EA680A85062BFF28E636F61C12E
:106930005FF163C15EF15F51260837E2FF0A03E1B0
:106940005E51100832E25F6B320E5E6F5FC160F124
:10695000616BAA6A100EA96E60C1A8FFA69CA69ED4
:10696000A684F250006EF29E0F01550EA76EAA0E7D
:10697000A76EA682A6B2FED7A6940050F212AA6A0B
:10698000110EA96E5EC1A8FFA69CA69EA684F2CF9A
:1069900000F0F29E550EA76EAA0EA76EA682A6B2B2
:1069A000FED7A6940050F21201015B515E5F000E0B
:1069B0005F5B5FC160F1616BAA6A100EA96E60C176
:1069C000A8FFA69CA69EA684F250006EF29E0F0120
:1069D000550EA76EAA0EA76EA682A6B2FED7A694E3
:1069E0000050F212AA6A110EA96E5EC1A8FFA69C01
:1069F000A69EA684F2CF00F0F29E550EA76EAA0EB8
:106A0000A76EA682A6B2FED7A6940050F212AC0ED4
:106A1000F66E2A0EF76E196AF2BE198EF29E00010A
:106A200082EC19F019BEF28E01015C530FE1B20E37
:106A3000F66E2A0EF76E196AF2BE198EF29E0001EA
:106A400082EC19F019BEF28E0ED00101BC0EF66E6A
:106A50002A0EF76E196AF2BE198EF29E000182ECC0
:106A600019F019BEF28ED80EF66E2A0EF76E196A5C
:106A7000F2BE198EF29E82EC19F019BEF28EF20E61
:106A8000F66E2A0EF76E196AF2BE198EF29E210E6C
:106A90000101BF6F00015DEC1AF019BEF28E100EFD
:106AA000E96E5FC170F15EC16FF132EC21F00A0E48
:106AB00004009EA8FDD7AD6E0D0E04009EA8FDD764
:106AC000AD6E080E0101606F196AF2BE198EF29E5A
:106AD000FA0EC26F000153EC1EF019BEF28E0101D6
:106AE000602FF2D70001000C01015081000188ECF9
:106AF00021F0015204E1B8EC22F0D0EF3BF0F1ECD0
:106B000023F0015204E1E6EC18F0D0EF3BF01B500B
:106B1000300803E21B50320804E21B506108D8A47D
:106B200020D10101586B576B58530FE1575173082F
:106B30000CE31D0E5725E96E000E5821EA6EFF0E7C
:106B4000EF6E572BD8B4582BEFD7586B740E576F86
:106B5000585100080BE31D0E5725E96E000E582111
:106B6000EA6EEF6A572BD8B4582BF2D7516B5151BC
:106B70002D081AE3036A51510001E5EC08F0036A9D
:106B80001D0FE96E000E0320EA6E036A01015151E8
:106B90002E0F016E000E032201500001E5EC08F0FB
:106BA000EF6E0101512BE3D74F3D80D0F2CF5BF167
:106BB000F29EAA6A320EA96EA69CA69EA680A85036
:106BC0005BBFF28E5A6B596F5A5303E159519708C4
:106BD00003E25A6B010E596F516B5151130859E37F
:106BE000036A515103C0F7FF00011BEC09F0036A6F
:106BF0001D0FE96E000E0320EA6E5AC15EF159C105
:106C00005DF10101606B140E5F6F00016EEC24F00A
:106C100002C05EF101C05DF1010151510124016E1C
:106C2000000E0220036E015003C0F7FF00011BECB1
:106C300009F0EF6E036A0101515103C0F7FF000133
:106C40001BEC09F0140F036A1D0FE96E000E032000
:106C5000EA6E5AC15EF159C15DF10101606B140E1B
:106C60005F6F00016EEC24F002C05EF101C05DF1C7
:106C7000010151510124016E000E0220036E0150EA
:106C800003C0F7FF00011BEC09F0EF6E0101512B6F
:106C9000A4D7592BD8B45A2B616B320E606F59C1EF
:106CA00062F10001E0EC20F05BD00101516B515129
:106CB00013082CE3036A515103C0F7FF00011BECDA
:106CC00009F0036A1D0FE96E000E0320EA6E010150
:106CD0005E6B4FC15DF1606B140E5F6F00016EEC77
:106CE00024F002C05EF101C05DF1010151510124A7
:106CF000016E000E0220036E015003C0F7FF000179
:106D00001BEC09F0EF6E0101512BD1D7036A5151F1
:106D100003C0F7FF00011BEC09F0140F036A1D0FFD
:106D2000E96E000E0320EA6E01015E6B4FC15DF15A
:106D3000606B140E5F6F00016EEC24F002C05EF118
:106D400001C05DF1010151510124016E000E0220CC
:106D5000036E015003C0F7FF00011BEC09F0EF6E5A
:106D60000CD20101586B576B585100080CE31D0EF3
:106D70005725E96E000E5821EA6EFF0EEF6E572B75
:106D8000D8B4582BF1D7516B51512D081AE3036A2F
:106D90005151000157EC04F0036A1D0FE96E000E1B
:106DA0000320EA6E036A010151512E0F016E000E9D
:106DB00003220150000157EC04F0EF6E0101512B4A
:106DC000E3D7010E4F5DFC0FD8B0D8D1040F0001FE
:106DD000D2EF3BF0F2CF5BF1F29EAA6A300EA96EC1
:106DE000A69CA69EA680A85001015BBFF28E5C6F98
:106DF000F2CF5DF1F29EAA6A310EA96EA69CA69E04
:106E0000A680A8505DBFF28E5E6F5CC15AF15EC174
:106E100059F15A5303E15951340803E25A6B010EF8
:106E2000596F516B515121082DE3036A515103C031
:106E3000F7FF00018DEC04F0036A1D0FE96E000EF0
:106E40000320EA6E5AC15EF159C15DF10101606B28
:106E5000220E5F6F00016EEC24F002C05EF101C0F3
:106E60005DF1010151510124016E000E0220036EFB
:106E7000015003C0F7FF00018DEC04F0EF6E01013B
:106E8000512BD0D7592BD8B45A2B5AC15BF15C6B1C
:106E9000616B300E606F5AC162F10001E0EC20F0CE
:106EA0000101616B310E606F59C162F10001E0ECCC
:106EB00020F0010163D1F2CF5BF1F29EAA6A320E9B
:106EC000A96EA69CA69EA680A85001015BBFF28E6B
:106ED0005C6FF2CF5DF1F29EAA6A330EA96EA69C9A
:106EE000A69EA680A8505DBFF28E5E6F5CC15AF16F
:106EF0005EC159F15A5308E159512F0805E35A531D
:106F000006E15951260803E35A6B270E596F516B5E
:106F1000515121082DE3036A515103C0F7FF0001CD
:106F20008DEC04F0036A1D0FE96E000E0320EA6E7B
:106F30005AC15EF159C15DF10101606B220E5F6FB4
:106F400000016EEC24F002C05EF101C05DF10101B0
:106F500051510124016E000E0220036E015003C046
:106F6000F7FF00018DEC04F0EF6E0101512BD0D73B
:106F7000592BD8B45A2B5AC15BF15C6B616B320E42
:106F8000606F5AC162F10001E0EC20F00101616B19
:106F9000330E606F59C162F10001E0EC20F0010195
:106FA000EDD0F2CF5BF1F29EAA6A340EA96EA69CD8
:106FB000A69EA680A85001015BBFF28E5C6FF2CF47
:106FC0005DF1F29EAA6A350EA96EA69CA69EA680C9
:106FD000A8505DBFF28E5E6F5CC15AF15EC159F17F
:106FE0005A5308E15951390805E35A5306E15951FA
:106FF0002F0803E35A6B2F0E596F516B5151210823
:107000002DE3036A515103C0F7FF00018DEC04F03A
:10701000036A1D0FE96E000E0320EA6E5AC15EF18D
:1070200059C15DF10101606B220E5F6F00016EECD2
:1070300024F002C05EF101C05DF101015151012453
:10704000016E000E0220036E015003C0F7FF000125
:107050008DEC04F0EF6E0101512BD0D7592BD8B431
:107060005A2B5AC15BF15C6B616B340E606F5AC175
:1070700062F10001E0EC20F00101616B350E606F00
:1070800059C162F10001E0EC20F0010177D0F2CFAC
:107090005BF1F29EAA6A360EA96EA69CA69EA680F9
:1070A000A85001015BBFF28E5C6FF2CF5DF1F29EE2
:1070B000AA6A370EA96EA69CA69EA680A8505DBFA0
:1070C000F28E5E6F5CC15AF15EC159F15A5308E10C
:1070D0005951410805E35A5306E15951390803E370
:1070E0005A6B3A0E596F516B515121082DE3036AC7
:1070F000515103C0F7FF00018DEC04F0036A1D0F2E
:10710000E96E000E0320EA6E5AC15EF159C15DF1CD
:107110000101606B220E5F6F00016EEC24F002C073
:107120005EF101C05DF1010151510124016E000EBB
:107130000220036E015003C0F7FF00018DEC04F044
:10714000EF6E0101512BD0D7592BD8B45A2B5AC10D
:107150005BF15C6B616B360E606F5AC162F10001CE
:10716000E0EC20F00101616B370E606F59C162F1F4
:107170000001E0EC20F0010101D001014FC142F01B
:107180004FC156F024C145F023C146F022C147F05B
:1071900021C148F024C159F023C15AF022C15BF04B
:1071A00021C15CF0310E1B5CCE0FD8B01ED1320F66
:1071B0000001E3EF3BF00101586B740E576F58511B
:1071C000000804E3572BD8B4582BF9D71D0E5725C8
:1071D000E96E000E5821EA6EEF6A010E416E556E9F
:1071E000110E446E586E01D10101586B740E576F29
:1071F0005851000804E3572BD8B4582BF9D71D0E6B
:107200005725E96E000E5821EA6EEF6A010E416EB5
:10721000556E110E446E586EE8D0010E416E556EDB
:107220000D0E446E586E01015B6B5D6B5C6B000173
:107230007FEC24F00101D9D0010E416E556E0D0E88
:10724000446E586E01015B6B5D6B5C6B00017FEC03
:1072500024F00101CAD0010E416E556E0D0E446E30
:10726000586E01015B6B5D6B5C6B00017FEC24F081
:107270000101BBD0010E416E556E0D0E446E586E6D
:1072800001015B6B5D6B5C6B00017FEC24F0010125
:10729000ACD0010E416E556E0D0E446E586E01015C
:1072A0005B6B5D6B5C6B00017FEC24F001019DD09A
:1072B000010E416E556E0D0E446E586E01015B6BF2
:1072C0005D6B5C6B00017FEC24F001018ED0020E3F
:1072D000416E556E110E446E586E01015B6B5D6B15
:1072E0005C6B00017FEC24F001017FD0020E416E47
:1072F000556E110E446E586E01015B6B5D6B5C6BDD
:1073000000017FEC24F0010170D0090E416E556E32
:10731000110E446E586E01015B6B5D6B5C6B00017E
:107320007FEC24F0010161D0090E416E556E110E03
:10733000446E586E01015B6B5D6B5C6B00017FEC12
:1073400024F0010152D0080E416E556E110E446EAC
:10735000586E01015B6B5D6B5C6B00017FEC24F090
:10736000010143D0080E416E556E0D0E446E586EED
:1073700001015B6B5D6B5C6B00017FEC24F0010134
:1073800034D0080E416E556E110E446E586E0101D8
:107390005B6B5D6B5C6B00017FEC24F0010125D021
:1073A0000D0E416E556E446E586E01015B6B5D6B48
:1073B0005C6B00017FEC24F0010117D0160E416ECA
:1073C000556E110E446E586E01010FD0010E416EC4
:1073D000556E110E446E586E01015B6B5D6B5C6BFC
:1073E00000017FEC24F0010100D00001E6EC18F070
:1073F000060EF66E240EF76E196AF2BE198EF29E14
:1074000082EC19F019BEF28E8E0EF66E2E0EF76E0D
:10741000196AF2BE198EF29E82EC19F019BEF28E34
:1074200027EC25F00101586B576B58510008D8A084
:10743000F8D0000151EC2AF0196AF2BE198EF29EC2
:10744000300E0101BD6F57C1BEF1BF6B000101ECF1
:107450001FF019BEF28E196AF2BE198EF29E01015A
:10746000BF6B000130EC1FF019BEF28E01C052F16B
:1074700093948A841D0E01015725E96E000E582150
:10748000EA6EEF50525DD8B4ACD0000151EC2AF056
:107490001D0E01015725E96E000E5821EA6EEFCF4F
:1074A0005BF1196AF2BE198EF29E380EBD6F57C19C
:1074B000BEF15BC1BFF1000101EC1FF019BEF28EFD
:1074C000CAEC22F069EC2AF01D0E01015725E96E85
:1074D000000E5821EA6EEFCF5BF157C179F1370EFC
:1074E0007A6F0001EAEC22F09D0EF66E2E0EF76E1A
:1074F000196AF2BE198EF29E090E0101BF6F0001DA
:107500005DEC1AF019BEF28E5BC179F1370E010104
:107510007A6F0001EAEC22F0A90EF66E2E0EF76EDD
:10752000196AF2BE198EF29E0B0E0101BF6F0001A7
:107530005DEC1AF019BEF28E51EC2AF01D0E01011D
:107540005725E96E000E5821EA6EEFCF5BF1196AFC
:10755000F2BE198EF29E300EBD6F57C1BEF15BC1F7
:10756000BFF1000101EC1FF019BEF28E196AF2BEE4
:10757000198EF29E0101BF6B000130EC1FF019BEA5
:10758000F28E01C052F193948A8452C179F1370E80
:1075900001017A6F0001EAEC22F00400A60E006EF1
:1075A000002EFED793948A941D0E01015725E96E93
:1075B000000E5821EA6EEF50525D12E05091B60E67
:1075C000F66E2E0EF76E196AF2BE198EF29E00014B
:1075D00082EC19F019BEF28EB8EC22F0E1D0010174
:1075E0001CD0000169EC2AF057C179F1370E010176
:1075F0007A6F0001EAEC22F0DF0EF66E2E0EF76EC7
:10760000196AF2BE198EF29E190E0101BF6F0001B8
:107610005DEC1AF019BEF28E0101572BD8B4582B2D
:1076200004D7FA0EF66E2E0EF76E196AF2BE198E98
:10763000F29E000182EC19F019BEF28E080E0101D3
:107640005B6F196AF2BE198EF29EFA0EC26F0001CC
:1076500053EC1EF019BEF28E01015B2FF2D75B6B6B
:107660005C6B5D6B0001C0EC2EF04AEC34F0015015
:107670004E081FE1840EF66E230EF76E196AF2BEF5
:10768000198EF29E82EC19F019BEF28E100E0101D5
:107690005B6F196AF2BE198EF29EFA0EC26F00017C
:1076A00053EC1EF019BEF28E01015B2FF2D70001E0
:1076B00077D01B50410803E01B50310809E101015C
:1076C000536B546BFF0E556F566F0AD009D00001F3
:1076D0000101536BF00E546F010E556FF00E566F93
:1076E000000151EC2AF00101586B576B585328E107
:1076F00057511F0825E353B11AD01D0E5725E96EC7
:10770000000E5821EA6EEFCF5BF1196AF2BE198EB6
:10771000F29E3C0EBD6F57C1BEF15BC1BFF10001CF
:1077200001EC1FF019BEF28ECAEC22F00101D890D4
:107730005633553354335333572BD8B4582BD6D7ED
:10774000196AF2BE198EF29E000160EC1FF019BE9C
:10775000F28EE6EC18F0D60EF66E230EF76E196A6E
:10776000F2BE198EF29E82EC19F019BEF28E010E55
:1077700001015B6F5C6B5D6B000174EC34F0080E13
:1077800001015B6F196AF2BE198EF29EFA0EC26F8A
:10779000000153EC1EF019BEF28E01015B2FF2D7EF
:1077A0000001000CE824F76AF736BF0FF66E770E7B
:1077B000F7220A00F550FA6E0800F550F96ED46D04
:1077C000B66EA26F8E70E824F76AF736E10FF66E98
:1077D000770EF7220A00F550FA6E0800F550F96EA0
:1077E000B671E8711A723872567274729272B0720F
:1077F000CE72EC720A732873467364738273A0733B
:10780000EA73EA73EA73EA73EA73EA73EA73EA7390
:10781000EA73EA73EA73EA73EA73EA73EA73EA7380
:10782000EA73EA73EA73EA73EA73EA73EA73EA7370
:10783000EA73EA73EA73EA73EA73EA73EA73EA7360
:10784000BC73CC73DEEC20F0196AF2BE198EF29E86
:1078500060EC1FF019BEF28E196AF2BE198EF29E0C
:10786000DBEC1CF019BEF28EF294F28AD180000C8F
:10787000196AF2BE198EF29E310E0101BD6FBE6B08
:10788000BF6B000101EC1FF019BEF28E0101536BBA
:10789000535103081EE3036A53514F0F016E010E4B
:1078A000032201C055F103C056F1196AF2BE198EC8
:1078B000F29E53C1BFF1000130EC1FF019BEF28EF1
:1078C00056C1EAFF55C1E9FF01C0EFFF0101532B8B
:1078D000DFD70001E6EC18F0520EF66E2E0EF76EB2
:1078E000196AF2BE198EF29E82EC19F019BEF28E60
:1078F00052C179F1370E01017A6F0001EAEC22F0F2
:10790000200E04009EA8FDD7AD6E51C179F1370E4F
:1079100001017A6F0001EAEC22F0200E04009EA81B
:10792000FDD7AD6E50C179F1370E01017A6F0001BC
:10793000EAEC22F0200E04009EA8FDD7AD6E4FC1E8
:1079400079F1370E01017A6F0001EAEC22F00D0E99
:1079500004009EA8FDD7AD6E0A0E04009EA8FDD7B8
:10796000AD6E0A0E04009EA8FDD7AD6E7E0EF66EBB
:107970002E0EF76E196AF2BE198EF29E82EC19F085
:1079800019BEF28E01014F51070B546F5451F80F7D
:10799000D8B06FD1080F00014DEF3EF0BA0EF66E71
:1079A000210EF76E196AF2BE198EF29E82EC19F062
:1079B00019BEF28EF00EF66E210EF76E196AF2BE47
:1079C000198EF29E82EC19F019BEF28E010151D18E
:1079D000700EF66E210EF76E196AF2BE198EF29EC7
:1079E0002B0E0101BF6F00015DEC1AF019BEF28E83
:1079F000196AF2BE198EF29E020E0101C06F1B0EB3
:107A0000C16F000111EC19F019BEF28E9D0EF66ED9
:107A1000210EF76E196AF2BE198EF29E1B0E01013D
:107A2000BF6F00015DEC1AF019BEF28E010121D189
:107A3000700EF66E210EF76E196AF2BE198EF29E66
:107A40002B0E0101BF6F00015DEC1AF019BEF28E22
:107A5000196AF2BE198EF29E020E0101C06F1B0E52
:107A6000C16F000111EC19F019BEF28E9D0EF66E79
:107A7000210EF76E196AF2BE198EF29E1B0E0101DD
:107A8000BF6F00015DEC1AF019BEF28E0101F1D05A
:107A9000700EF66E210EF76E196AF2BE198EF29E06
:107AA0002B0E0101BF6F00015DEC1AF019BEF28EC2
:107AB000196AF2BE198EF29E020E0101C06F1B0EF2
:107AC000C16F000111EC19F019BEF28E9D0EF66E19
:107AD000210EF76E196AF2BE198EF29E1B0E01017D
:107AE000BF6F00015DEC1AF019BEF28E0101C1D02A
:107AF000700EF66E210EF76E196AF2BE198EF29EA6
:107B00002B0E0101BF6F00015DEC1AF019BEF28E61
:107B1000196AF2BE198EF29E010E0101C06F1B0E92
:107B2000C16F000111EC19F019BEF28E9D0EF66EB8
:107B3000210EF76E196AF2BE198EF29E1B0E01011C
:107B4000BF6F00015DEC1AF019BEF28E010191D0F9
:107B5000700EF66E210EF76E196AF2BE198EF29E45
:107B60002B0E0101BF6F00015DEC1AF019BEF28E01
:107B7000196AF2BE198EF29E010E0101C06F1B0E32
:107B8000C16F000111EC19F019BEF28E9D0EF66E58
:107B9000210EF76E196AF2BE198EF29E1B0E0101BC
:107BA000BF6F00015DEC1AF019BEF28E010161D0C9
:107BB000700EF66E210EF76E196AF2BE198EF29EE5
:107BC0002B0E0101BF6F00015DEC1AF019BEF28EA1
:107BD000196AF2BE198EF29E010E0101C06F1B0ED2
:107BE000C16F000111EC19F019BEF28E9D0EF66EF8
:107BF000210EF76E196AF2BE198EF29E1B0E01015C
:107C0000BF6F00015DEC1AF019BEF28E010131D098
:107C1000700EF66E210EF76E196AF2BE198EF29E84
:107C20002B0E0101BF6F00015DEC1AF019BEF28E40
:107C3000196AF2BE198EF29E030E0101C06F1B0E6F
:107C4000C16F000111EC19F019BEF28E9D0EF66E97
:107C5000210EF76E196AF2BE198EF29E1B0E0101FB
:107C6000BF6F00015DEC1AF019BEF28E010101D068
:107C700001010D0E04009EA8FDD7AD6E0A0E040092
:107C80009EA8FDD7AD6E0A0E04009EA8FDD7AD6E6E
:107C90000001B8EC22F02BEF5BF0E824F76AF7362E
:107CA000B50FF66E7C0EF7220A00F550FA6E08004A
:107CB000F550F96E9C79F07A507BD079B07B307AB0
:107CC000907A107CDEEC20F0196AF2BE198EF29EDA
:107CD00060EC1FF019BEF28E196AF2BE198EF29E88
:107CE000DBEC1CF019BEF28EF294F28AD180000C0B
:107CF00004009EA8FDD7AD6E000C01017207736BE6
:107D000004009EAAFDD7AECF74F1745108080EE1AD
:107D100073530BE0730774510001EADF200EE8DFB4
:107D2000010174510001E4DF010117D074511F08F3
:107D300014E274517E0811E37351725D0EE37351C6
:107D4000732B036A7025E96E71510320EA6E74C1CA
:107D5000EFFF74510001CCDF010174510D08D0E137
:107D6000036A73517025E96E71510320EA6EEF6A60
:107D70000001E8EF3FF0010179517B19800B7D6F25
:107D800079AF05D0781F791F782BD8B4792B7BAFCA
:107D900005D07A1F7B1F7A2BD8B47B2B78517A03BE
:107DA000F3CF01F0F4CF00F07B03F35000267951BC
:107DB0007A03F3500020026E7DAF05D0011E021E33
:107DC000012AD8B4022A000159EF3FF00101766B75
:107DD000746B0A0E756F736B726B7051711104E1E5
:107DE000000E016E026EE8D07651762B036A702584
:107DF000E96E71510320EA6EEFCF77F177512D08CC
:107E00000DE1010E746F7651762B036A7025E96ED1
:107E100071510320EA6EEFCF77F10DD077512B0827
:107E20000AE17651762B036A7025E96E71510320C1
:107E3000EA6EEFCF77F177512F08D8B0AFD07751F6
:107E40003908D8A0ABD07751300821E1036A7651C8
:107E50007025E96E71510320EA6EEF5078080AE050
:107E6000036A76517025E96E71510320EA6EEF5076
:107E700058080DE1100E756F762B7651762B036A3C
:107E80007025E96E71510320EA6EEFCF77F17551DD
:107E90000A0823E177512F081FE2775139081CE3C4
:107EA000796B0A0E786F73C17BF172C17AF10001B0
:107EB00062D7300E0101775D0124726F000E02203F
:107EC000736F7651762B036A7025E96E715103202A
:107ED000EA6EEFCF77F1DED761D0755110085EE121
:107EE0007751600806E277517A0803E37751DF0B98
:107EF00001D07751776F77512F0803E27751390816
:107F000006E2775140084AE27751460847E3775145
:107F10002F0819E27751390816E37235786F7335F7
:107F2000796F783779377837793778377937F00E4E
:107F30007817300E775D7825016E000E792101C02B
:107F400072F1736F16D07235786F7335796F783739
:107F500079377837793778377937F00E7817410ED7
:107F6000775D0A0F7825016E000E792101C072F14C
:107F7000736F7651762B036A7025E96E7151032079
:107F8000EA6EEF50776F600806E277517A0803E3F4
:107F90007751DF0B01D07751776FADD775510A0854
:107FA00007E1742D05D0721F731F722BD8B4732B89
:107FB00072C101F073C102F00001EFEF3FF0010E5A
:107FC0000101716F670E706F070E726F000195D619
:107FD000010E0101716F670E706F0001F7D602C0CC
:107FE0006FF101C06EF101016EC101F06FC102F0CD
:107FF0000001000C010E0101BA6FBA51B95D07E32F
:10800000B531B833B733B633B533BA2BF6D7B5C1BC
:1080100000F0B6C101F0B7C102F0B8C103F0000131
:10802000000C010E0101BA6FBA51B95D07E3B83512
:10803000B537B637B737B837BA2BF6D7B5C100F072
:10804000B6C101F0B7C102F0B8C103F00001000CE5
:10805000120E0101726F340E716F560E706F780E32
:108060006F6F010E6D6F6D510A0839E36D51040D8C
:10807000F350036A6F0F016E010E032201C0AFF1CE
:1080800003C0B0F1010E6D5D040DF350036A6F0F74
:10809000E96E010E0320EA6EEFCFB1F1ECCFB2F141
:1080A000ECCFB3F1ECCFB4F1B4C1B8F1B3C1B7F1D7
:1080B000B2C1B6F1B1C1B5F1020EB96F00019ADFDC
:1080C000B0C1EAFFAFC1E9FF00C0EFFF01C0ECFFA4
:1080D00002C0ECFF03C0ECFF01016D2BC4D7F2CF4F
:1080E000AFF1F29EAA6A200EA96EA69CA69EA6805B
:1080F000A850AFBFF28EB06FF2CFB1F1F29EAA6A74
:10810000210EA96EA69CA69EA680A850B1BFF28E95
:10811000B26F67C19DF168C19EF1B0C19CF1B2C15F
:108120009BF19A0EA26FBC0EA16FDE0EA06FF00E37
:108130009F6FF2CFAFF1F29EAA6A220EA96EA69CA3
:10814000A69EA680A850AFBFF28EB06FB0C1A6F1B8
:10815000FF0EA56FFF0EA46F800EA36FAA6BA96B15
:10816000A86BA76BAE6BAD6B010EAC6FB80EAB6FAF
:10817000670E366F450E356F230E346F010E336F69
:10818000EF0E3A6FCD0E396FAB0E386F890E376F29
:10819000980E3E6FBA0E3D6FDC0E3C6FFE0E3B6FCD
:1081A000100E426F320E416F540E406F760E3F6FCD
:1081B000C30E466FD20E456FE10E446FF00E436F53
:1081C0006D6B6D514F08D8A0BBD26D510F0B6E6F08
:1081D0006D510F08D8B087D06E51040DF350036A6B
:1081E0006F0F016E010E032201C0AFF103C0B0F1A9
:1081F0000D0E6E250F0B040DF350036A6F0FE96E21
:10820000010E0320EA6EEFCFB1F1ECCFB2F1ECCF6B
:10821000B3F1ECCFB4F1080E6E250F0B040DF35043
:10822000036A6F0FE96E010E0320EA6EEFCF00F0D4
:10823000ECCF01F0ECCF02F0ECCF03F00050B11B1B
:108240000150B21B0250B31B0350B41B020E6E252B
:108250000F0B040DF350036A6F0FE96E010E03203C
:10826000EA6EEFCF00F0ECCF01F0ECCF02F0ECCFF4
:1082700003F00050B11B0150B21B0250B31B03505E
:10828000B41B6E51040DF350036A6F0FE96E010EBB
:108290000320EA6EEFCF00F0ECCF01F0ECCF02F05C
:1082A000ECCF03F00050B11B0150B21B0250B31BC6
:1082B0000350B41BB4C1B8F1B3C1B7F1B2C1B6F148
:1082C000B1C1B5F1010EB96F0001ABDEB0C1EAFF7B
:1082D000AFC1E9FF00C0EFFF01C0ECFF02C0ECFF3F
:1082E00003C0ECFF01016D51130802E2000E01D042
:1082F000010E010B7AE036C1B8F135C1B7F134C1D6
:10830000B6F133C1B5F1050EB96F00018ADE03C0C5
:10831000B2F102C0B1F101C0B0F100C0AFF1010192
:1083200037513B15B36F38513C15B46F39513D157A
:10833000B56F3A513E15B66F37C1B7F1B71F38C1A7
:10834000B8F1B81F39C1B9F1B91F3AC1BAF1BA1FB2
:10835000B7513F15006EB8514015016EB951411526
:10836000026EBA514215036E0050B311006E0150F7
:10837000B411016E0250B511026E0350B611036EB6
:108380000050AF270150B0230250B1230350B22355
:108390004351AF274451B0234551B1234651B22335
:1083A0006E51040DF350036A6F0FE96E010E032046
:1083B000EA6EEFCF00F0ECCF01F0ECCF02F0ECCFA3
:1083C00003F00050AF270150B0230250B1230350F7
:1083D000B223990EAF25696F790EB0216A6F820EB4
:1083E000B1216B6F5A0EB2216C6F6D51130802E30D
:1083F000000E01D0010EAF6F6D51270802E2000E92
:1084000001D0010EAF1562E036C1B8F135C1B7F148
:1084100034C1B6F133C1B5F1050EB96F000101DE0B
:1084200003C0B2F102C0B1F101C0B0F100C0AFF1C0
:10843000010137513B19B36F38513C19B46F3951B1
:108440003D19B56F3A513E19B66FB3513F19006EE1
:10845000B4514019016EB5514119026EB65142191D
:10846000036E0050AF270150B0230250B1230350D8
:10847000B2234351AF274451B0234551B123465154
:10848000B2236E51040DF350036A6F0FE96E010EB3
:108490000320EA6EEFCF00F0ECCF01F0ECCF02F05A
:1084A000ECCF03F00050AF270150B0230250B123AE
:1084B0000350B223A10EAF25696FEB0EB0216A6F96
:1084C000D90EB1216B6F6E0EB2216C6F6D51270802
:1084D00002E3000E01D0010EAF6F6D513B0802E2C6
:1084E000000E01D0010EAF15D8B482D036C1B8F15C
:1084F00035C1B7F134C1B6F133C1B5F1050EB96F6D
:1085000000018FDD03C0B2F102C0B1F101C0B0F1D2
:1085100000C0AFF1010137513B15B36F38513C1525
:10852000B46F39513D15B56F3A513E15B66F37519D
:108530003F15006E38514015016E39514115026EDC
:108540003A514215036E0050B3130150B413025058
:10855000B5130350B6133B513F15006E3C51401507
:10856000016E3D514115026E3E514215036E0050A1
:10857000B311006E0150B411016E0250B511026EBC
:108580000350B611036E0050AF270150B0230250C4
:10859000B1230350B2234351AF274451B023455177
:1085A000B1234651B2236E51040DF350036A6F0F8D
:1085B000E96E010E0320EA6EEFCF00F0ECCF01F080
:1085C000ECCF02F0ECCF03F00050AF270150B02306
:1085D0000250B1230350B223DC0EAF25696FBC0EED
:1085E000B0216A6F1B0EB1216B6F8F0EB2216C6FC1
:1085F0006D513B0802E3000E01D0010EAF6F6D51CB
:108600004F0802E2000E01D0010EAF1562E036C144
:10861000B8F135C1B7F134C1B6F133C1B5F1050ECA
:10862000B96F0001FEDC03C0B2F102C0B1F101C0BC
:10863000B0F100C0AFF1010137513B19B36F3851B0
:108640003C19B46F39513D19B56F3A513E19B66FA7
:10865000B3513F19006EB4514019016EB551411923
:10866000026EB6514219036E0050AF270150B0237D
:108670000250B1230350B2234351AF274451B023DA
:108680004551B1234651B2236E51040DF350036A94
:108690006F0FE96E010E0320EA6EEFCF00F0ECCF12
:1086A00001F0ECCF02F0ECCF03F00050AF27015007
:1086B000B0230250B1230350B223D60EAF25696F09
:1086C000C10EB0216A6F620EB1216B6FCA0EB2216A
:1086D0006C6F42C146F141C145F140C144F13FC117
:1086E00043F13EC142F13DC141F13CC140F13BC1CA
:1086F0003FF13AC1B8F139C1B7F138C1B6F137C16C
:10870000B5F1020EB96F000175DC03C03EF102C085
:108710003DF101C03CF100C03BF136C13AF135C139
:1087200039F134C138F133C137F16CC136F16BC165
:1087300035F16AC134F169C133F101016D2B41D5C5
:108740000001CAEF44F004009EAAFDD7AECF6CF141
:1087500001016C51000178EC3EF001016C513908C7
:1087600005E3300E6C5D016E0FD00ED06C516008C9
:1087700006E26C517A0803E36C51DF0B01D06C51B7
:10878000BF0F0A0F016E00D00001000CDCDF01C03A
:108790006BF1D9DF01C06AF101016A51DD0804E122
:1087A0006BC101F007D006D06B51100DF3506A2554
:1087B000016E00D00001000CE6EC18F0F2CF67F17A
:1087C000F29EAA6A200EA96EA69CA69EA680A8501C
:1087D000010167BFF28E686FF2CF69F1F29EAA6A5B
:1087E000210EA96EA69CA69EA680A85069BFF28EF7
:1087F0006A6F68C16CF16AC16BF1F2CF6DF1F29EE4
:10880000AA6A220EA96EA69CA69EA680A8506DBF3D
:10881000F28E6E6F160EF66E290EF76E196AF2BEA4
:10882000198EF29E150EBF6F00015DEC1AF019BE95
:10883000F28E100EE96E6CC170F16BC16FF132EC0B
:1088400021F02E0EF66E290EF76E196AF2BE198E01
:10885000F29E0D0E0101BF6F00015DEC1AF019BE12
:10886000F28E196AF2BE198EF29E6EC1C0F11B0E15
:108870000101C16F000111EC19F019BEF28E0D0E4D
:1088800004009EA8FDD7AD6E0A0E04009EA8FDD779
:10889000AD6E0A0E04009EA8FDD7AD6E420EF66EB8
:1088A000290EF76E196AF2BE198EF29E82EC19F04B
:1088B00019BEF28E900EF66E290EF76E196AF2BE90
:1088C000198EF29E82EC19F019BEF28EF2CF67F18A
:1088D000F29EAA6A100EA96EA69CA69EA680A8501B
:1088E000010167BFF28E686FF2CF69F1F29EAA6A4A
:1088F000110EA96EA69CA69EA680A85069BFF28EF6
:108900006A6F68C152F16AC151F1DE0EF66E290E2E
:10891000F76E196AF2BE198EF29E130EBF6F000138
:108920005DEC1AF019BEF28E100EE96E52C170F1B4
:1089300051C16FF132EC21F00D0E04009EA8FDD75D
:10894000AD6E0A0E04009EA8FDD7AD6E0A0E04009F
:108950009EA8FDD7AD6EF80EF66E290EF76E196A59
:10896000F2BE198EF29E82EC19F019BEF28EDFEC87
:108970003FF002C050F101C04FF101014F5303E13C
:10898000505301E182D150C168F14FC167F100013C
:1089900028EF40F0300EF66E2A0EF76E196AF2BE1E
:1089A000198EF29E82EC19F019BEF28E040EF66E4C
:1089B000260EF76E196AF2BE198EF29E82EC19F03D
:1089C00019BEF28E5E0EF66E2A0EF76E196AF2BEB0
:1089D000198EF29E82EC19F019BEF28ED7DE01C01C
:1089E00067F1D4DE01C068F1D1DE01C069F1CEDEED
:1089F00067C156F168C155F169C154F101C053F125
:108A0000C5DE01C067F1C2DE01C068F1BFDE01C092
:108A100069F1BCDE67C15AF168C159F169C158F109
:108A200001C057F1B3DE01C067F1B0DE01C068F1EB
:108A3000ADDE01C069F1AADE67C15EF168C15DF11A
:108A400069C15CF101C05BF1A1DE01C067F19EDE8E
:108A500001C068F19BDE01C069F198DE67C162F177
:108A600068C161F169C160F101C05FF18FDE01C0D1
:108A700067F18CDE01C068F189DE01C069F186DE34
:108A800067C166F168C165F169C164F101C063F154
:108A900001013351535DD8A4DAD03451545DD8A4C8
:108AA000D6D03551555DD8A4D2D03651565DD8A414
:108AB000CED03751575DD8A4CAD03851585DD8A40C
:108AC000C6D03951595DD8A4C2D03A515A5DD8A404
:108AD000BED03B515B5DD8A4BAD03C515C5DD8A4FC
:108AE000B6D03D515D5DD8A4B2D03E515E5DD8A4F4
:108AF000AED03F515F5DD8A4AAD04051605DD8A4EC
:108B0000A6D04151615DD8A4A2D04251625DD8A4E3
:108B10009ED04351635DD8A49AD04451645DD8A4DB
:108B200096D04551655DD8A492D04651665DD8A4D3
:108B30008ED051514F275251502350C167F1686B6D
:108B4000AA6A100EA96E67C1A8FFA69CA69EA6845D
:108B5000F250006EF29E0F01550EA76EAA0EA76E80
:108B6000A682A6B2FED7A6940050F212AA6A110EEF
:108B7000A96E4FC1A8FFA69CA69EA684F2CF00F0C6
:108B8000F29E550EA76EAA0EA76EA682A6B2FED7BB
:108B9000A6940050F212F2CF67F1F29EAA6A220E5A
:108BA000A96EA69CA69EA680A850010167BFF28E62
:108BB000010F686FAA6A220EA96E68C1A8FFA69C61
:108BC000A69EA684F250006EF29E0F01550EA76E6F
:108BD000AA0EA76EA682A6B2FED7A6940050F212E5
:108BE000640EF66E2A0EF76E196AF2BE198EF29EA8
:108BF0002B0E0101BF6F00015DEC1AF019BEF28E61
:108C0000100EE96E52C170F151C16FF132EC21F0DA
:108C1000920EF66E2A0EF76E196AF2BE198EF29E49
:108C2000040E0101BF6F00015DEC1AF019BEF28E57
:108C3000100EE96E50C170F14FC16FF132EC21F0AE
:108C40002E0E04009EA8FDD7AD6E0ED001019C0E25
:108C5000F66E2A0EF76E196AF2BE198EF29E0001A8
:108C600082EC19F019BEF28E080E0101676F196AC5
:108C7000F2BE198EF29EFA0EC26F000153EC1EF086
:108C800019BEF28E0101672FF2D7000132EF5BF0BF
:108C900001015B6B5C6B010E5D6F0001C0EC2EF09F
:108CA0000D0E04009EA8FDD7AD6E0A0E04009EA80E
:108CB000FDD7AD6E196AF2BE198EF29E380E010113
:108CC000BD6F4FC1BEF151C1BFF1000101EC1FF0FA
:108CD00019BEF28ECAEC22F0196AF2BE198EF29E0B
:108CE000010E0101C26F000153EC1EF019BEF28E9D
:108CF00001015B6B5C6B010E5D6F0001C0EC2EF03F
:108D0000196AF2BE198EF29E300E0101BD6F4FC17D
:108D1000BEF1BF6B000101EC1FF019BEF28E196AA3
:108D2000F2BE198EF29E0101BF6B000130EC1FF004
:108D300019BEF28E01C052F193948A840400A60EEB
:108D4000006E002EFED793948A940D0E04009EA808
:108D5000FDD7AD6E0A0E04009EA8FDD7AD6E0101D1
:108D60005151525D17E1900EF66E300EF76E196A92
:108D7000F2BE198EF29E000182EC19F019BEF28E3D
:108D8000010E01015B6F5C6B5D6B000174EC34F0F4
:108D900030D00101A60EF66E300EF76E196AF2BEE3
:108DA000198EF29E200EBF6F00015DEC1AF019BE05
:108DB000F28E51C179F1370E01017A6F0001EAECB0
:108DC00022F0C90EF66E300EF76E196AF2BE198ED9
:108DD000F29E060E0101BF6F00015DEC1AF019BE94
:108DE000F28E52C179F1370E01017A6F0001EAEC7F
:108DF00022F075EF5BF00101606B616B010E626F39
:108E0000DA6AD96A656F580E646F010EEA6E5C0EFD
:108E1000E96E65C1E2FF64C1E1FF62C163F1D89010
:108E2000E550EE02F3506023F4506123632FF7D72F
:108E300060C1DEFF61C160F1616BD8B0612B642B52
:108E4000D8B4652B622B62510508DFE10001000CEC
:108E50000101536B526B535100081BE352C158F18F
:108E6000010E5325596F1D0E5225E96E000E532138
:108E7000EA6EEFCF5AF159C161F152C160F15AC1A6
:108E800062F10001E0EC20F00101522BD8B4532B29
:108E9000E2D70001E6EC18F0180EF66E2F0EF76E12
:108EA000196AF2BE198EF29E82EC19F019BEF28E8A
:108EB00004009EAAFDD7AECF4FF101014F516008CB
:108EC00006E24F517A0803E34F51DF0B01D04F51B7
:108ED0004F6F4F51580803E04F51520801E103D042
:108EE0000001DAD701010D0E04009EA8FDD7AD6E7A
:108EF0000A0E04009EA8FDD7AD6E0A0E04009EA8BF
:108F0000FDD7AD6E4F515208D8A47ED2010E616FCD
:108F10001C0E606FFF0E626F0001E0EC20F0010E8E
:108F20000101616F1D0E606FFF0E626F0001E0ECCA
:108F300020F0010E0101616F1E0E606FFF0E626F67
:108F40000001E0EC20F0010E0101616F1F0E606F67
:108F5000FF0E626F0001E0EC20F02C0E0101516F5A
:108F600051512F080DE351C158F1010E616F51C1EC
:108F700060F1626B0001E0EC20F00101512BF0D7B1
:108F8000400E516F515146080DE351C158F1010E89
:108F9000616F51C160F1626B0001E0EC20F00101F2
:108FA000512BF0D70001E6EC18F0196AF2BE198EC9
:108FB000F29E010E0101BD6F250EBE6F280EBF6F20
:108FC000000153EC19F019BEF28E3C0EF66E2F0E16
:108FD000F76E196AF2BE198EF29E82EC19F019BE74
:108FE000F28E196AF2BE198EF29E94EC19F019BE37
:108FF000F28E640EF66E2F0EF76E196AF2BE198E9F
:10900000F29E82EC19F019BEF28E8C0EF66E2F0EC7
:10901000F76E196AF2BE198EF29E82EC19F019BE33
:10902000F28EDFEC3FF001C000F002C001F0026AF6
:10903000036A03C057F102C056F101C055F100C0E8
:1090400054F1010157530AE1565308E155510F08F5
:1090500008E2FF0A03E15451C60803E20001D5D734
:10906000010155C159F154C158F1010E5B6F55C151
:109070005DF154C15CF100017FEC24F06D0E040041
:109080009EA8FDD7AD6E6C0E04009EA8FDD7AD6EF8
:1090900057C15BF156C15AF155C159F154C158F14C
:1090A00001015F6B0F0E5E6F420E5D6F400E5C6FD5
:1090B0000001A1DE03C057F102C056F101C055F115
:1090C00000C054F157C159F101015A6B5B6B5C6BE5
:1090D000010E616F280E606F57C162F10001E0EC74
:1090E00020F056C159F157C15AF101015B6B5C6B1D
:1090F000010E616F290E606F56C162F10001E0EC54
:1091000020F055C159F156C15AF157C15BF1010127
:109110005C6B010E616F2A0E606F55C162F1000138
:10912000E0EC20F0010E0101616F2B0E606F54C165
:1091300062F10001E0EC20F057C159F101015A6BD6
:109140005B6B5C6B010E616F3C0E606F57C162F12F
:109150000001E0EC20F056C159F157C15AF101016C
:109160005B6B5C6B010E616F3D0E606F56C162F10F
:109170000001E0EC20F055C159F156C15AF157C138
:109180005BF101015C6B010E616F3E0E606F55C1BA
:1091900062F10001E0EC20F0010E0101616F3F0E71
:1091A000606F54C162F10001E0EC20F00D0E04008C
:1091B0009EA8FDD7AD6E0A0E04009EA8FDD7AD6E29
:1091C0000A0E04009EA8FDD7AD6E200E04009EA8D6
:1091D000FDD7AD6E120EF66E1E0EF76E196AF2BE58
:1091E000198EF29E410E0101BF6F00015DEC1AF075
:1091F00019BEF28E200E04009EA8FDD7AD6E0D0E96
:1092000004009EA8FDD7AD6E0A0E04009EA8FDD7EF
:10921000AD6E200E04009EA8FDD7AD6E5A0EF66E00
:109220001E0EF76E196AF2BE198EF29E410E0101F2
:10923000BF6F00015DEC1AF019BEF28E200E040023
:109240009EA8FDD7AD6E0D0E04009EA8FDD7AD6E95
:109250000A0E04009EA8FDD7AD6E200E04009EA845
:10926000FDD7AD6EA20EF66E1E0EF76E196AF2BE37
:10927000198EF29E410E0101BF6F00015DEC1AF0E4
:1092800019BEF28E200E04009EA8FDD7AD6E0D0E05
:1092900004009EA8FDD7AD6E0A0E04009EA8FDD75F
:1092A000AD6EBA0EF66E2F0EF76E196AF2BE198EFB
:1092B000F29E82EC19F019BEF28EA3EC43F001C0CD
:1092C00050F101015051060803E200016FD701017E
:1092D000010E505DFA0FD8B089D0060F00014FEF94
:1092E0004AF0010E0101616F250E606F010E626F81
:1092F0000001E0EC20F0010E0101616F390E606F9A
:10930000010E626F0001E0EC20F001016FD0010E50
:109310000101616F250E606F020E626F0001E0ECCB
:1093200020F0010E0101616F390E606F020E626F55
:109330000001E0EC20F0010159D0010E0101616F44
:10934000250E606F030E626F0001E0EC20F0010E4D
:109350000101616F390E606F030E626F0001E0EC76
:1093600020F0010143D0010E0101616F250E606FF5
:10937000040E626F0001E0EC20F0010E0101616F4C
:10938000390E606F040E626F0001E0EC20F0010105
:109390002DD0010E0101616F250E606F050E626F09
:1093A0000001E0EC20F0010E0101616F390E606FE9
:1093B000050E626F0001E0EC20F0010117D0010EF4
:1093C0000101616F250E606F060E626F0001E0EC17
:1093D00020F0010E0101616F390E606F060E626FA1
:1093E0000001E0EC20F0010101D00101D80EF66E81
:1093F0002F0EF76E196AF2BE198EF29E000182ECF2
:1094000019F019BEF28E0101010E5B6F5C6B5D6B92
:109410000001C0EC2EF00D0E04009EA8FDD7AD6E2D
:109420000A0E04009EA8FDD7AD6E010E0101766FF5
:10943000776B00010FEC23F00101536B526B535318
:109440001FE1525103081CE3F00E5225586F000E25
:109450005321596F1D0E5225E96E010E5321EA6EFC
:10946000EFCF5AF159C161F158C160F15AC162F1AF
:109470000001E0EC20F00101522BD8B4532BDFD7D0
:10948000FA0EF66E2F0EF76E196AF2BE198EF29E64
:10949000000182EC19F019BEF28EAAEF5BF0E8240D
:1094A000F76AF736B90FF66E940EF7220A00F550F8
:1094B000FA6E0800F550F96EE2920E933A936693B5
:1094C0009293BE9301014F81000188EC21F001527B
:1094D00003E1B8EC22F0A4D2F1EC23F0015201E157
:1094E0009FD227EC25F051EC2AF0060EF66E240EE2
:1094F000F76E196AF2BE198EF29E82EC19F019BE4F
:10950000F28E240EF66E300EF76E196AF2BE198EC8
:10951000F29E82EC19F019BEF28E27EC25F00101C3
:10952000566B556B56510008D8A01BD1000151EC69
:109530002AF0196AF2BE198EF29E300E0101BD6F3B
:1095400055C1BEF1BF6B000101EC1FF019BEF28ED8
:10955000196AF2BE198EF29E0101BF6B000130EC58
:109560001FF019BEF28E01C050F193948A8401015C
:109570005551576F010E5625586FF2CF59F1F29E93
:1095800058C1AAFF57C1A9FFA69CA69EA680A850B5
:1095900059BFF28E505DD8B4C4D0000151EC2AF00E
:1095A00001015551576F010E5625586FF2CF59F1F1
:1095B000F29E58C1AAFF57C1A9FFA69CA69EA680ED
:1095C000A85059BFF28E576F196AF2BE198EF29EDB
:1095D000380EBD6F55C1BEF157C1BFF1000101EC9E
:1095E0001FF019BEF28ECAEC22F069EC2AF00101DC
:1095F0005551576F010E5625586FF2CF59F1F29E13
:1096000058C1AAFF57C1A9FFA69CA69EA680A85034
:1096100059BFF28E576F55C179F1370E7A6F00013D
:10962000EAEC22F0330EF66E300EF76E196AF2BED7
:10963000198EF29E090E0101BF6F00015DEC1AF058
:1096400019BEF28E57C179F1370E01017A6F000110
:10965000EAEC22F03F0EF66E300EF76E196AF2BE9B
:10966000198EF29E0B0E0101BF6F00015DEC1AF026
:1096700019BEF28E51EC2AF0196AF2BE198EF29ED2
:10968000300E0101BD6F55C1BEF1BF6B000101EC91
:109690001FF019BEF28E196AF2BE198EF29E0101F8
:1096A000BF6B000130EC1FF019BEF28E01C050F10B
:1096B00093948A8450C179F1370E01017A6F0001C9
:1096C000EAEC22F00400A60E006E002EFED7939462
:1096D0008A9401015551576F010E5625586FF2CFEC
:1096E00059F1F29E58C1AAFF57C1A9FFA69CA69E98
:1096F000A680A85059BFF28E505D12E04F914C0EDB
:10970000F66E300EF76E196AF2BE198EF29E0001E7
:1097100082EC19F019BEF28EB8EC22F081D1010171
:109720001CD0000169EC2AF055C179F1370E010116
:109730007A6F0001EAEC22F0750EF66E300EF76ECD
:10974000196AF2BE198EF29E190E0101BF6F000157
:109750005DEC1AF019BEF28E0101552BD8B4562BD0
:10976000E1D6196AF2BE198EF29E000160EC1FF07C
:1097700019BEF28E196AF2BE198EF29E320E0101E6
:10978000C26F000153EC1EF019BEF28E196AF2BED0
:10979000198EF29E6BEC1EF019BEF28E196AF2BEA3
:1097A000198EF29E73EC1EF019BEF28E68EC1FF05B
:1097B0000101566B040E556F56510008D8A09AD07F
:1097C000196AF2BE198EF29E300EBD6F55C1BEF100
:1097D000BF6B000101EC1FF019BEF28E1D0E0101DE
:1097E0005525016E000E5621036E01C057F1586FCA
:1097F000196AF2BE198EF29EBF6B000130EC1FF0A9
:1098000019BEF28E58C1EAFF57C1E9FF01C0EFFF50
:10981000010E01015525576F000E5621586F1D0E80
:109820005725016E000E5821036E01C057F1586F85
:10983000196AF2BE198EF29E010EBF6F000130EC64
:109840001FF019BEF28E58C1EAFF57C1E9FF01C0EF
:10985000EFFF020E01015525576F000E5621586F7C
:109860001D0E5725016E000E5821036E01C057F1E1
:10987000586F196AF2BE198EF29E010EBF6F000179
:1098800030EC1FF019BEF28E58C1EAFF57C1E9FF54
:1098900001C0EFFF030E01015525576F000E562141
:1098A000586F1D0E5725016E000E5821036E01C022
:1098B00057F1586F196AF2BE198EF29E010EBF6FF2
:1098C000000130EC1FF019BEF28E58C1EAFF57C1FB
:1098D000E9FF01C0EFFF93948A840400A60E006E96
:1098E000002EFED793948A94040E01015527000E92
:1098F000562362D7196AF2BE198EF29E000160ECFF
:109900001FF019BEF28E01015B6B5C6B5D6B000199
:10991000C0EC2EF04AEC34F001504E0801E180D04A
:109920000101566B556B565321E1555103081EE357
:10993000510E5525E96E010E5621EA6EF00E5525A1
:10994000596F000E56215A6FF2CF5BF1F29E5AC149
:10995000AAFF59C1A9FFA69CA69EA680A8505BBFDE
:10996000F28EEF6E552BD8B4562BDDD7000151EC9B
:109970002AF00101566B556B565333E155511F08C0
:1099800030E351B125D05551576F010E5625586F10
:10999000F2CF59F1F29E58C1AAFF57C1A9FFA69C68
:1099A000A69EA680A85059BFF28E576F196AF2BEC4
:1099B000198EF29E3C0EBD6F55C1BEF157C1BFF16D
:1099C000000101EC1FF019BEF28ECAEC22F0010179
:1099D000D8905433533352335133552BD8B4562B7C
:1099E000CBD7196AF2BE198EF29E000160EC1FF00F
:1099F00019BEF28EE6EC18F0D60EF66E230EF76E58
:109A0000196AF2BE198EF29E82EC19F019BEF28E1E
:109A1000010E01015B6F5C6F5D6B000174EC34F053
:109A2000B9EF5BF0E4EF5BF0010150810001E6EC7F
:109A300018F0196AF2BE198EF29E010E0101BD6F77
:109A4000250EBE6F280EBF6F000153EC19F019BE32
:109A5000F28ED40EF66E300EF76E196AF2BE198EC3
:109A6000F29E82EC19F019BEF28E196AF2BE198EBE
:109A7000F29E94EC19F019BEF28EEE0EF66E300ED8
:109A8000F76E196AF2BE198EF29E82EC19F019BEB9
:109A9000F28E080EF66E310EF76E196AF2BE198E4E
:109AA000F29E82EC19F019BEF28E196AF2BE198E7E
:109AB000F29E010E0101BD6F250EBE6F280EBF6F15
:109AC000000153EC19F019BEF28EA80EF66E240EAA
:109AD000F76E196AF2BE198EF29E82EC19F019BE69
:109AE000F28E196AF2BE198EF29E94EC19F019BE2C
:109AF000F28E0D0E04009EA8FDD7AD6E0A0E040076
:109B00009EA8FDD7AD6E0E0EF66E310EF76E196A79
:109B1000F2BE198EF29E82EC19F019BEF28E196A0D
:109B2000F2BE198EF29E010E0101BD6F250EBE6FB1
:109B3000280EBF6F000153EC19F019BEF28EBE0E55
:109B4000F66E240EF76E196AF2BE198EF29E82EC42
:109B500019F019BEF28E196AF2BE198EF29E94ECBB
:109B600019F019BEF28E0D0E04009EA8FDD7AD6E41
:109B70000A0E04009EA8FDD7AD6E140EF66E310ECF
:109B8000F76E196AF2BE198EF29E82EC19F019BEB8
:109B9000F28E196AF2BE198EF29E010E0101BD6F9E
:109BA000250EBE6F280EBF6F000153EC19F019BED1
:109BB000F28ED80EF66E240EF76E196AF2BE198E6A
:109BC000F29E82EC19F019BEF28E196AF2BE198E5D
:109BD000F29E94EC19F019BEF28E0D0E04009EA8B0
:109BE000FDD7AD6E0A0E04009EA8FDD7AD6E1A0E0D
:109BF000F66E310EF76E196AF2BE198EF29E82EC85
:109C000019F019BEF28E196AF2BE198EF29E010E7B
:109C10000101BD6F250EBE6F280EBF6F000153EC12
:109C200019F019BEF28EF20EF66E240EF76E196A56
:109C3000F2BE198EF29E82EC19F019BEF28E196AEC
:109C4000F2BE198EF29E94EC19F019BEF28E0D0E32
:109C500004009EA8FDD7AD6E0A0E04009EA8FDD795
:109C6000AD6E200EF66E310EF76E196AF2BE198EC9
:109C7000F29E82EC19F019BEF28E196AF2BE198EAC
:109C8000F29E010E0101BD6F250EBE6F280EBF6F43
:109C9000000153EC19F019BEF28E060EF66E250E79
:109CA000F76E196AF2BE198EF29E82EC19F019BE97
:109CB000F28E196AF2BE198EF29E94EC19F019BE5A
:109CC000F28E0D0E04009EA8FDD7AD6E0A0E0400A4
:109CD0009EA8FDD7AD6E260EF66E310EF76E196A90
:109CE000F2BE198EF29E82EC19F019BEF28E196A3C
:109CF000F2BE198EF29E010E0101BD6F250EBE6FE0
:109D0000280EBF6F000153EC19F019BEF28E180E29
:109D1000F66E250EF76E196AF2BE198EF29E82EC6F
:109D200019F019BEF28E196AF2BE198EF29E94ECE9
:109D300019F019BEF28E0D0E04009EA8FDD7AD6E6F
:109D40000A0E04009EA8FDD7AD6E2C0EF66E310EE5
:109D5000F76E196AF2BE198EF29E82EC19F019BEE6
:109D6000F28E196AF2BE198EF29E010E0101BD6FCC
:109D7000250EBE6F280EBF6F000153EC19F019BEFF
:109D8000F28E2E0EF66E250EF76E196AF2BE198E41
:109D9000F29E82EC19F019BEF28E196AF2BE198E8B
:109DA000F29E94EC19F019BEF28E0D0E04009EA8DE
:109DB000FDD7AD6E0A0E04009EA8FDD7AD6E320E23
:109DC000F66E310EF76E196AF2BE198EF29E82ECB3
:109DD00019F019BEF28E196AF2BE198EF29E010EAA
:109DE0000101BD6F250EBE6F280EBF6F000153EC41
:109DF00019F019BEF28E3E0EF66E250EF76E196A38
:109E0000F2BE198EF29E82EC19F019BEF28E196A1A
:109E1000F2BE198EF29E94EC19F019BEF28E0D0E60
:109E200004009EA8FDD7AD6E0A0E04009EA8FDD7C3
:109E3000AD6E380EF66E310EF76E196AF2BE198EDF
:109E4000F29E82EC19F019BEF28E196AF2BE198EDA
:109E5000F29E010E0101BD6F250EBE6F280EBF6F71
:109E6000000153EC19F019BEF28E520EF66E250E5B
:109E7000F76E196AF2BE198EF29E82EC19F019BEC5
:109E8000F28E196AF2BE198EF29E94EC19F019BE88
:109E9000F28E0D0E04009EA8FDD7AD6E0A0E0400D2
:109EA0009EA8FDD7AD6E3E0EF66E310EF76E196AA6
:109EB000F2BE198EF29E82EC19F019BEF28E196A6A
:109EC000F2BE198EF29E010E0101BD6F250EBE6F0E
:109ED000280EBF6F000153EC19F019BEF28E620E0E
:109EE000F66E250EF76E196AF2BE198EF29E82EC9E
:109EF00019F019BEF28E196AF2BE198EF29E94EC18
:109F000019F019BEF28E0D0E04009EA8FDD7AD6E9D
:109F10000A0E04009EA8FDD7AD6E440EF66E310EFB
:109F2000F76E196AF2BE198EF29E82EC19F019BE14
:109F3000F28E196AF2BE198EF29E010E0101BD6FFA
:109F4000250EBE6F280EBF6F000153EC19F019BE2D
:109F5000F28E760EF66E250EF76E196AF2BE198E27
:109F6000F29E82EC19F019BEF28E196AF2BE198EB9
:109F7000F29E94EC19F019BEF28E0D0E04009EA80C
:109F8000FDD7AD6E0A0E04009EA8FDD7AD6E4A0E39
:109F9000F66E310EF76E196AF2BE198EF29E82ECE1
:109FA00019F019BEF28E196AF2BE198EF29E010ED8
:109FB0000101BD6F250EBE6F280EBF6F000153EC6F
:109FC00019F019BEF28E800EF66E250EF76E196A24
:109FD000F2BE198EF29E82EC19F019BEF28E196A49
:109FE000F2BE198EF29E94EC19F019BEF28E0D0E8F
:109FF00004009EA8FDD7AD6E0A0E04009EA8FDD7F2
:10A00000AD6E500EF66E310EF76E196AF2BE198EF5
:10A01000F29E82EC19F019BEF28E196AF2BE198E08
:10A02000F29E010E0101BD6F250EBE6F280EBF6F9F
:10A03000000153EC19F019BEF28E900EF66E250E4B
:10A04000F76E196AF2BE198EF29E82EC19F019BEF3
:10A05000F28E196AF2BE198EF29E94EC19F019BEB6
:10A06000F28E0D0E04009EA8FDD7AD6E0A0E040000
:10A070009EA8FDD7AD6E560EF66E310EF76E196ABC
:10A08000F2BE198EF29E82EC19F019BEF28E196A98
:10A09000F2BE198EF29E010E0101BD6F250EBE6F3C
:10A0A000280EBF6F000153EC19F019BEF28E9C0E02
:10A0B000F66E250EF76E196AF2BE198EF29E82ECCC
:10A0C00019F019BEF28E196AF2BE198EF29E94EC46
:10A0D00019F019BEF28E0D0E04009EA8FDD7AD6ECC
:10A0E0000A0E04009EA8FDD7AD6E5C0EF66E310E12
:10A0F000F76E196AF2BE198EF29E82EC19F019BE43
:10A10000F28E196AF2BE198EF29E010E0101BD6F28
:10A11000250EBE6F280EBF6F000153EC19F019BE5B
:10A12000F28EAC0EF66E250EF76E196AF2BE198E1F
:10A13000F29E82EC19F019BEF28E196AF2BE198EE7
:10A14000F29E94EC19F019BEF28E0D0E04009EA83A
:10A15000FDD7AD6E0A0E04009EA8FDD7AD6E620E4F
:10A16000F66E310EF76E196AF2BE198EF29E82EC0F
:10A1700019F019BEF28E196AF2BE198EF29E010E06
:10A180000101BD6F250EBE6F280EBF6F000153EC9D
:10A1900019F019BEF28EC20EF66E250EF76E196A10
:10A1A000F2BE198EF29E82EC19F019BEF28E196A77
:10A1B000F2BE198EF29E94EC19F019BEF28E0D0EBD
:10A1C00004009EA8FDD7AD6E0A0E04009EA8FDD720
:10A1D000AD6E680EF66E310EF76E196AF2BE198E0C
:10A1E000F29E82EC19F019BEF28E196AF2BE198E37
:10A1F000F29E010E0101BD6F250EBE6F280EBF6FCE
:10A20000000153EC19F019BEF28EDA0EF66E250E2F
:10A21000F76E196AF2BE198EF29E82EC19F019BE21
:10A22000F28E196AF2BE198EF29E94EC19F019BEE4
:10A23000F28E0D0E04009EA8FDD7AD6E0A0E04002E
:10A240009EA8FDD7AD6E6E0EF66E310EF76E196AD2
:10A25000F2BE198EF29E82EC19F019BEF28E196AC6
:10A26000F2BE198EF29E010E0101BD6F250EBE6F6A
:10A27000280EBF6F000153EC19F019BEF28EE80EE4
:10A28000F66E250EF76E196AF2BE198EF29E82ECFA
:10A2900019F019BEF28E196AF2BE198EF29E94EC74
:10A2A00019F019BEF28E0D0E04009EA8FDD7AD6EFA
:10A2B0000A0E04009EA8FDD7AD6E0A0E04009EA8EB
:10A2C000FDD7AD6E740EF66E310EF76E196AF2BEE2
:10A2D000198EF29E82EC19F019BEF28E04009EAA2D
:10A2E000FDD7AECF4FF101014F51300804E24F517D
:10A2F000390801E34AD04F51600806E24F517A080D
:10A3000003E34F51DF0B01D04F514F6F4F51410AC3
:10A31000000111E0030A13E0010A15E0070A17E043
:10A32000010A19E0030A1BE0010A1DE00F0A1FE001
:10A33000010A21E024D03A0E01014F6F22D03B0EDA
:10A3400001014F6F1ED03C0E01014F6F1AD03D0E20
:10A3500001014F6F16D03E0E01014F6F12D03F0E1C
:10A3600001014F6F0ED0400E01014F6F0AD0610EF8
:10A3700001014F6F06D0620E01014F6F02D0010143
:10A38000509150B102D015EF4DF04FC11BF00001BC
:10A39000E6EC18F0980EF66E310EF76E196AF2BE02
:10A3A000198EF29E82EC19F019BEF28E196AF2BE75
:10A3B000198EF29E010E0101BD6F250EBE6F280E93
:10A3C000BF6F000153EC19F019BEF28E310E01017E
:10A3D0004F5DCE0FD8B001D1320F00013CEF57F0E6
:10A3E000A80EF66E240EF76E196AF2BE198EF29E52
:10A3F00082EC19F019BEF28E0101EFD0BE0EF66E9E
:10A40000240EF76E196AF2BE198EF29E82EC19F0D4
:10A4100019BEF28E0101E1D0060EF66E250EF76E22
:10A42000196AF2BE198EF29E82EC19F019BEF28EF4
:10A430000101D3D0180EF66E250EF76E196AF2BE22
:10A44000198EF29E82EC19F019BEF28E0101C5D070
:10A450002E0EF66E250EF76E196AF2BE198EF29E5A
:10A4600082EC19F019BEF28E0101B7D03E0EF66EE5
:10A47000250EF76E196AF2BE198EF29E82EC19F063
:10A4800019BEF28E0101A9D0520EF66E250EF76E9E
:10A49000196AF2BE198EF29E82EC19F019BEF28E84
:10A4A00001019BD0620EF66E250EF76E196AF2BEA0
:10A4B000198EF29E82EC19F019BEF28E01018DD038
:10A4C000760EF66E250EF76E196AF2BE198EF29EA2
:10A4D00082EC19F019BEF28E01017FD0800EF66E6B
:10A4E000250EF76E196AF2BE198EF29E82EC19F0F3
:10A4F00019BEF28E010171D0900EF66E250EF76E28
:10A50000196AF2BE198EF29E82EC19F019BEF28E13
:10A51000010163D09C0EF66E250EF76E196AF2BE2D
:10A52000198EF29E82EC19F019BEF28E010155D0FF
:10A53000AC0EF66E250EF76E196AF2BE198EF29EFB
:10A5400082EC19F019BEF28E010147D0C20EF66EF0
:10A55000250EF76E196AF2BE198EF29E82EC19F082
:10A5600019BEF28E010139D0DA0EF66E250EF76EA5
:10A57000196AF2BE198EF29E82EC19F019BEF28EA3
:10A5800001012BD0E80EF66E250EF76E196AF2BEA9
:10A59000198EF29E82EC19F019BEF28E01011DD0C7
:10A5A000D80EF66E240EF76E196AF2BE198EF29E60
:10A5B00082EC19F019BEF28E01010FD0F20EF66E88
:10A5C000240EF76E196AF2BE198EF29E82EC19F013
:10A5D00019BEF28E010101D00101196AF2BE198E75
:10A5E000F29E000194EC19F019BEF28E0D0E0400DB
:10A5F0009EA8FDD7AD6E0A0E04009EA8FDD7AD6ED5
:10A600000A0E04009EA8FDD7AD6EAC0EF66E310E9C
:10A61000F76E196AF2BE198EF29E82EC19F019BE1D
:10A62000F28E310E1B5CCE0FD8B0E0EF56F0320F39
:10A630007BEF57F0FA0EF66E220EF76E196AF2BE35
:10A64000198EF29E82EC19F019BEF28E04009EAAB9
:10A65000FDD7AECF4FF101014F51310A000103E0A8
:10A66000030A08E00FD00101246B236B226BDC0E80
:10A67000216F0FD00101246B236B010E226FB80EE6
:10A68000216F07D00101246B236B010E226FB80EDE
:10A69000216F0001E0EF56F00C0EF66E230EF76E00
:10A6A000196AF2BE198EF29E82EC19F019BEF28E72
:10A6B00004009EAAFDD7AECF4FF101014F51310AE0
:10A6C000000103E0030A09E010D00101246B236BB1
:10A6D000030E226F700E216F0FD00101246B236BCC
:10A6E000030E226FE80E216F07D00101246B236B4C
:10A6F000030E226FE80E216F0001E0EF56F0FA0E14
:10A70000F66E220EF76E196AF2BE198EF29E82EC78
:10A7100019F019BEF28E04009EAAFDD7AECF4FF1FC
:10A7200001014F51310A000103E0030A08E00FD094
:10A730000101246B236B226BDC0E216F0FD0010112
:10A74000246B236B010E226FB80E216F07D001011D
:10A75000246B236B010E226FB80E216F0001E0EF16
:10A7600056F0200EF66E230EF76E196AF2BE198EA1
:10A77000F29E82EC19F019BEF28EDFEC3FF001C0C0
:10A7800000F002C001F0026A036A03C024F102C0B3
:10A7900023F101C022F100C021F10101215306E1A2
:10A7A000225304E1235302E124530CE024530AE131
:10A7B000235308E122510F080BE2FF0A03E1215164
:10A7C000C70806E2246B236B030E226FE80E216F8D
:10A7D0000001F6D2FA0EF66E220EF76E196AF2BE7C
:10A7E000198EF29E82EC19F019BEF28E04009EAA18
:10A7F000FDD7AECF4FF101014F51310A000103E007
:10A80000030A08E00FD00101246B236B226BDC0EDE
:10A81000216F0FD00101246B236B010E226FB80E44
:10A82000216F07D00101246B236B010E226FB80E3C
:10A83000216F0001C5D2200EF66E230EF76E196A45
:10A84000F2BE198EF29E82EC19F019BEF28EDFEC88
:10A850003FF001C000F002C001F0026A036A03C0C9
:10A8600024F102C023F101C022F100C021F1010155
:10A87000215306E1225304E1235302E124530CE067
:10A8800024530AE1235308E122510F080BE2FF0A87
:10A8900003E12151C70806E2246B236B030E226FEC
:10A8A000E80E216F00018CD2FA0EF66E220EF76EC2
:10A8B000196AF2BE198EF29E82EC19F019BEF28E60
:10A8C00004009EAAFDD7AECF4FF101014F51310ACE
:10A8D000000103E0030A08E00FD00101246B236BA1
:10A8E000226BDC0E216F0FD00101246B236B010E54
:10A8F000226FB80E216F07D00101246B236B010E6C
:10A90000226FB80E216F00015BD2200EF66E230E6F
:10A91000F76E196AF2BE198EF29E82EC19F019BE1A
:10A92000F28EDFEC3FF001C000F002C001F0026ADD
:10A93000036A03C024F102C023F101C022F100C068
:10A9400021F10101215306E1225304E1235302E1E5
:10A9500024530CE024530AE1235308E122510F0849
:10A960000BE2FF0A03E12151C70806E2246B236BC7
:10A97000030E226FE80E216F000122D2FA0EF66E4E
:10A98000220EF76E196AF2BE198EF29E82EC19F051
:10A9900019BEF28E04009EAAFDD7AECF4FF1010181
:10A9A0004F51310A000103E0030A08E00FD0010112
:10A9B000246B236B226BDC0E216F0FD00101246B03
:10A9C000236B010E226FB80E216F07D00101246B9B
:10A9D000236B010E226FB80E216F0001F1D1200E02
:10A9E000F66E230EF76E196AF2BE198EF29E82EC95
:10A9F00019F019BEF28EDFEC3FF001C000F002C08A
:10AA000001F0026A036A03C024F102C023F101C00D
:10AA100022F100C021F10101215306E1225304E19A
:10AA2000235302E124530CE024530AE1235308E1A9
:10AA300022510F080BE2FF0A03E12151C70806E289
:10AA4000246B236B070E226FD00E216F0001B8D14B
:10AA5000FA0EF66E220EF76E196AF2BE198EF29E8B
:10AA600082EC19F019BEF28E04009EAAFDD7AECF7B
:10AA70004FF101014F51310A000103E0030A08E0E0
:10AA80000FD00101246B236B226BDC0E216F0FD0E2
:10AA90000101246B236B010E226FB80E216F07D0CA
:10AAA0000101246B236B010E226FB80E216F000190
:10AAB00087D1200EF66E230EF76E196AF2BE198E3C
:10AAC000F29E82EC19F019BEF28EDFEC3FF001C06D
:10AAD00000F002C001F0026A036A03C024F102C060
:10AAE00023F101C022F100C021F10101215306E14F
:10AAF000225304E1235302E124530CE024530AE1DE
:10AB0000235308E122510F080BE2FF0A03E1215110
:10AB1000C70806E2246B236B030E226FE80E216F39
:10AB200000014ED1FA0EF66E220EF76E196AF2BED1
:10AB3000198EF29E82EC19F019BEF28E04009EAAC4
:10AB4000FDD7AECF4FF101014F51310A000103E0B3
:10AB5000030A08E00FD00101246B236B226BDC0E8B
:10AB6000216F0FD00101246B236B010E226FB80EF1
:10AB7000216F07D00101246B236B010E226FB80EE9
:10AB8000216F00011DD1200EF66E230EF76E196A9B
:10AB9000F2BE198EF29E82EC19F019BEF28EDFEC35
:10ABA0003FF001C000F002C001F0026A036A03C076
:10ABB00024F102C023F101C022F100C021F1010102
:10ABC000215306E1225304E1235302E124530CE014
:10ABD00024530AE1235308E122510F080BE2FF0A34
:10ABE00003E12151C70806E2246B236B030E226F99
:10ABF000E80E216F0001E4D0200EF66E230EF76EF2
:10AC0000196AF2BE198EF29E82EC19F019BEF28E0C
:10AC1000DFEC3FF001C000F002C001F0026A036AFD
:10AC200003C024F102C023F101C022F100C021F1D0
:10AC30000101215306E1225304E1235302E124538D
:10AC40000CE024530AE1235308E122510F080BE2E0
:10AC5000FF0A03E12151C70806E2246B236B030EB0
:10AC6000226FE80E216F0001ABD0200EF66E230E8E
:10AC7000F76E196AF2BE198EF29E82EC19F019BEB7
:10AC8000F28EDFEC3FF001C000F002C001F0026A7A
:10AC9000036A03C024F102C023F101C022F100C005
:10ACA00021F10101215306E1225304E1235302E182
:10ACB00024530CE024530AE1235308E122510F08E6
:10ACC0000BE2FF0A03E12151C70806E2246B236B64
:10ACD000030E226FE80E216F000172D0200EF66E77
:10ACE000230EF76E196AF2BE198EF29E82EC19F0ED
:10ACF00019BEF28EDFEC3FF001C000F002C001F09F
:10AD0000026A036A03C024F102C023F101C022F1E8
:10AD100000C021F10101215306E1225304E1235334
:10AD200002E124530CE024530AE1235308E12251A9
:10AD30000F080BE2FF0A03E12151C70806E2246B6A
:10AD4000236B0F0E226FA00E216F000139D0200E51
:10AD5000F66E230EF76E196AF2BE198EF29E82EC21
:10AD600019F019BEF28EDFEC3FF001C000F002C016
:10AD700001F0026A036A03C024F102C023F101C09A
:10AD800022F100C021F10101215306E1225304E127
:10AD9000235302E124530CE024530AE1235308E136
:10ADA00022510F080BE2FF0A03E12151C70806E216
:10ADB000246B236B010E226FB80E216F000100D0AF
:10ADC00024C15BF123C15AF122C159F121C158F1CB
:10ADD00001015F6B0F0E5E6F420E5D6F400E5C6F88
:10ADE0000001FBEC46F003C024F102C023F101C0D6
:10ADF00022F100C021F10101616B130E606F1BC0D5
:10AE000062F10001E0EC20F024C152F10101536B2A
:10AE1000546B556B616B140E606F24C162F10001BD
:10AE2000E0EC20F023C152F124C153F10101546B35
:10AE3000556B616B150E606F23C162F10001E0EC90
:10AE400020F022C152F123C153F124C154F1010178
:10AE5000556B616B160E606F22C162F10001E0EC70
:10AE600020F00101616B170E606F21C162F10001DA
:10AE7000E0EC20F0EBEF5BF0E824F76AF736930F95
:10AE8000F66EAE0EF7220A00F550FA6E0800F55085
:10AE9000F96EE0A3FCA318A434A450A46CA488A465
:10AEA000A4A4C0A4DCA4F8A414A530A54CA568A54E
:10AEB00084A5D8A5D8A5D8A5D8A5D8A5D8A5D8A5FE
:10AEC000D8A5D8A5D8A5D8A5D8A5D8A5D8A5D8A59A
:10AED000D8A5D8A5D8A5D8A5D8A5D8A5D8A5D8A58A
:10AEE000D8A5D8A5D8A5D8A5D8A5D8A5D8A5D8A57A
:10AEF000D8A5A0A5BCA5E824F76AF736110FF66E11
:10AF0000AF0EF7220A00F550FA6E0800F550F96E00
:10AF100034A698A6FEA662A7D4A736A8A8A80AA910
:10AF20007CA9DEA950AAB2AA24AB86ABF8AB6AAC66
:10AF3000C0ADC0ADC0ADC0ADC0ADC0ADC0ADC0ADA9
:10AF4000C0ADC0ADC0ADC0ADC0ADC0ADC0ADC0AD99
:10AF5000C0ADC0ADC0ADC0ADC0ADC0ADC0ADC0AD89
:10AF6000C0ADC0ADC0ADC0ADC0ADC0ADC0ADC0AD79
:10AF7000DCAC4EADF86AD09E078EEA6AE96AB88604
:10AF80002A0EAF6E000EB06EA60EAC6E900EAB6EBB
:10AF90001A90FF0E0101286F276F266F256F2C6F07
:10AFA0002B6F2A6F296FC150C00B0F09C16E070E9E
:10AFB000B46E2D6B2E6BC150C00B0F09C16EC290C9
:10AFC000C69A949A94889496010EC66E000EC76E27
:10AFD000D190810ED56ECD6A000ECA6E000ECB6E7A
:10AFE000070EB46E9250926E0400100E006E002E8A
:10AFF000FED7B450A19CB56AF19E0001D5EF20F0B8
:10B0000068EC1FF0196AF2BE198EF29EC80E01019B
:10B01000C26F000153EC1EF019BEF28EDEEC20F080
:10B02000F2CF4FF1F29EAA6A130EA96EA69CA69EBD
:10B03000A680A85001014FBFF28E1B6E1B50300836
:10B0400003E21B50620849E2310E1B6E616B130E66
:10B05000606F1CC062F10001E0EC20F01A0E0101EB
:10B06000246F390E236FDE0E226F216B24C150F145
:10B07000516B526B536B616B140E606F24C162F1A4
:10B080000001E0EC20F023C150F124C151F1010195
:10B09000526B536B616B150E606F23C162F100013F
:10B0A000E0EC20F022C150F123C151F124C152F152
:10B0B0000101536B616B140E606F22C162F10001DC
:10B0C000E0EC20F00101616B150E606F21C162F1AF
:10B0D0000001E0EC20F081D00101F2CF4FF1F29EAF
:10B0E000AA6A140EA96EA69CA69EA680A8504FBF61
:10B0F000F28E506FF2CF51F1F29EAA6A150EA96E30
:10B10000A69CA69EA680A85051BFF28E526FF2CF89
:10B1100053F1F29EAA6A160EA96EA69CA69EA68060
:10B12000A85053BFF28E546FF2CF55F1F29EAA6A27
:10B13000170EA96EA69CA69EA680A85055BFF28E9B
:10B14000566F50C124F152C123F154C122F156C1AE
:10B1500021F1213D43D0223D41D0233D3FD0243D2C
:10B160003DD01A0E246F390E236FDE0E226F216B35
:10B1700024C150F1516B526B536B616B140E606FB5
:10B1800024C162F10001E0EC20F023C150F124C1A0
:10B1900051F10101526B536B616B150E606F23C14E
:10B1A00062F10001E0EC20F022C150F123C151F125
:10B1B00024C152F10101536B616B140E606F22C107
:10B1C00062F10001E0EC20F00101616B150E606F8F
:10B1D00021C162F10001E0EC20F0010193881A9294
:10B1E00081B81A82F2CF4FF1F29EAA6A300EA96E90
:10B1F000A69CA69EA680A8504FBFF28E506FF2CF9D
:10B2000051F1F29EAA6A310EA96EA69CA69EA68056
:10B21000A85051BFF28E526F50C14EF152C14DF144
:10B220004E5303E14D51340818E24E6B010E4D6F41
:10B230004EC14FF1506B616B300E606F4EC162F1C9
:10B240000001E0EC20F00101616B310E606F4DC137
:10B2500062F10001E0EC20F00101F2CF4FF1F29E2B
:10B26000AA6A320EA96EA69CA69EA680A8504FBFC1
:10B27000F28E506FF2CF51F1F29EAA6A330EA96E90
:10B28000A69CA69EA680A85051BFF28E526F50C1B8
:10B290004EF152C14DF14E5308E14D512F0805E3D7
:10B2A0004E531FE14D5126081CE34D51270802E182
:10B2B0004E5302E0000E00D04EC14FF1506B616B57
:10B2C000320E606F4EC162F10001E0EC20F001012E
:10B2D000616B330E606F4DC162F10001E0EC20F054
:10B2E0000101F2CF4FF1F29EAA6A340EA96EA69C1C
:10B2F000A69EA680A8504FBFF28E506FF2CF51F19C
:10B30000F29EAA6A350EA96EA69CA69EA680A8509B
:10B3100051BFF28E526F50C103F052514D5D03E1A7
:10B3200003504E5D02E0000E00D04E5308E14D5137
:10B33000390805E34E531FE14D512F081CE34D51D1
:10B34000300802E14E5302E0000E00D04EC14FF132
:10B35000506B616B340E606F4EC162F10001E0EC26
:10B3600020F00101616B350E606F4DC162F100018B
:10B37000E0EC20F00101F2CF4FF1F29EAA6A360E06
:10B38000A96EA69CA69EA680A8504FBFF28E506FB5
:10B39000F2CF51F1F29EAA6A370EA96EA69CA69E24
:10B3A000A680A85051BFF28E526F50C103F0525187
:10B3B0004D5D03E103504E5D02E0000E00D04E53A0
:10B3C00008E14D51410805E34E531EE14D51390846
:10B3D0001BE34D513A0802E14E5302E0000E00D04B
:10B3E0004EC14FF1506B616B360E606F4EC162F112
:10B3F0000001E0EC20F00101616B370E606F4DC180
:10B4000062F10001E0EC20F00001F9EF20F005EF1F
:10B4100021F0196AF2BE198EF29EDBEC1CF019BE07
:10B42000F28ED76AD66AF294F28AC00EF212D180F6
:10B4300004009EAAFDD7AECF48F101014851600833
:10B4400006E248517A0803E34851DF0B01D0485126
:10B45000486F040EF66E410EF76E196AF2BE198E31
:10B46000F29E120EBF6F00015DEC1AF019BEF28E53
:10B470000101485104009EA8FDD7AD6E0D0E0400D9
:10B480009EA8FDD7AD6E0A0E04009EA8FDD7AD6E36
:10B490004851310A000134E0030A40E0010A4CE05F
:10B4A000070A58E0010AD8B463D0030AD8B46ED0B2
:10B4B000010AD8B479D07A0AD8B491D01D0AD8B488
:10B4C0009FD0030AD8B4BDD0010AD8B4C7D0070AA8
:10B4D000D8B4CBD0020AD8B40BD1160AD8B430D124
:10B4E000030AD8B43CD10C0AD8B446D10A0AD8B45D
:10B4F00061D1070AD8B46BD10A0AD8B46FD178D118
:10B50000938881B801D07DD1F29A010E01014F6F6D
:10B51000000174EC35F022EC3CF073D1938881B8D3
:10B5200001D06FD1F29A020E01014F6F000174EC4D
:10B5300035F022EC3CF065D1938881B801D061D11F
:10B54000F29A030E01014F6F000174EC35F022EC0A
:10B550003CF057D1938881B801D053D1F29A040EB0
:10B5600001014F6F000174EC35F022EC3CF049D141
:10B57000938881B801D045D1F29A050E01014F6F31
:10B58000000174EC35F022EC3CF03BD1938881B89B
:10B5900001D037D1F29A060E01014F6F000174EC11
:10B5A00035F022EC3CF02DD1938881B801D029D11F
:10B5B000F29A1B50310803E01B50320807E1FF0EDE
:10B5C00001014F6F000174EC35F006D0FE0E010151
:10B5D0004F6F000174EC35F022EC3CF012D19388EF
:10B5E00081B801D00ED1F29AD19001015B6B010EAE
:10B5F0005C6F5D6F0001C0EC2EF022EC3CF001D1DD
:10B60000938881B801D0FDD0F29A0D0E04009EA857
:10B61000FDD7AD6E0A0E04009EA8FDD7AD6E0A0ED2
:10B6200004009EA8FDD7AD6ED190010E0101766F8A
:10B63000776F00010FEC23F0B8EC22F022EC3CF025
:10B64000E0D0938881B801D0DCD0F29AD19051EC4F
:10B650002AF038EF3CF062EC3EF0D3D0F29AD19071
:10B66000DCEF43F022EC3CF0CCD0938881B801D0E1
:10B67000C8D01AB001D0C5D0F29AD1901C0EF66E87
:10B68000410EF76E196AF2BE198EF29E82EC19F025
:10B6900019BEF28EC6EC43F001C047F10D0E040056
:10B6A0009EA8FDD7AD6E0A0E04009EA8FDD7AD6E14
:10B6B000500EF66E410EF76E196AF2BE198EF29EAA
:10B6C00082EC19F019BEF28EC6EC43F001014E6B0C
:10B6D00001C04DF1000151EC2AF04EC150F14DC1B5
:10B6E0004FF147C151F148EF46F022EC3CF089D0D0
:10B6F000938881B801D085D01AB001D082D0F29A57
:10B70000D1907C0EF66E410EF76E196AF2BE198E5C
:10B71000F29E82EC19F019BEF28EC6EC43F001C025
:10B7200049F1C6EC43F001C04AF1C6EC43F001C058
:10B730004BF1C6EC43F001C04CF122EC3CF061D07F
:10B74000938881B801D05DD0F29AD19051EC2AF063
:10B7500028EF47F0B8EC22F062EC3EF052D093882C
:10B7600081B801D04ED0F29AD19051EC2AF062EF1C
:10B770004AF062EC3EF045D0F29AD190010E010100
:10B780005B6F5C6B5D6B0001C0EC2EF00D0E040076
:10B790009EA8FDD7AD6E0A0E04009EA8FDD7AD6E23
:10B7A0000A0E04009EA8FDD7AD6EB8EC22F062EC44
:10B7B0003EF027D0938881B801D023D0F29AD1905F
:10B7C00051EC2AF012EF4DF062EC3EF01AD0F29AF2
:10B7D000D19014EF4DF022EC3CF013D01A70196A9E
:10B7E000F2BE198EF29EDBEC1CF019BEF28E09D06F
:10B7F000196AF2BE198EF29EDBEC1CF019BEF28EB5
:06B8000000D016D6030083
:020000040030CA
:0E00000000C20E1E00858100000007A0070050
:00000001FF
